:020000040000fa
:080000000002040000000000f2
:020000040000fa
:100400002f8f21000e7f24000e01880000000000c5
:100410000c000700a00023000100200011000700cd
:10042000000020000000e000020032000000020096
:10043000000000001a3c0200000000000040da004a
:100440000000fe004440a900204e20000000e00013
:100450000300320000002000a00188004440a800f2
:100460000000060091018800800078000000eb0089
:1004700015003700e280400032a0b4009101ba00bc
:10048000e280400032a0b4009102ba00e280400055
:1004900032a0b4000002eb00472bde00f507b200eb
:1004a000602ce10004003a000059eb008301e900f0
:1004b000fdff3e00040037006128e100010032002a
:1004c0000082eb00040007001101ba000200e00006
:1004d000e8ff3a00000006003159ba008301e90044
:1004e0000c0032002159ba008301e90008003200f3
:1004f0000400e00003003a00e280400032a0b400b3
:10050000f5ff370011d9ba008301e900faff3a007c
:100510008100e800e180400032a0b4000000060045
:10052000541e040000000000641e040000000000cf
:10053000741e0400000000002a1f040000000000d8
:1005400048200400000000002e21040000000000ec
:10055000841e040000000000b61e0400000000001d
:10056000c21e040000000000d21e040000000000b3
:10057000e01e0400000000003e2104000000000016
:10058000ce210400000000009422040000000000be
:10059000c022040000000000b0230400000000009e
:1005a000f4230400000000005e23040000000000ab
:1005b000082404000000000068240400000000007b
:1005c0008c24040000000000a024040000000000af
:1005d000fa240400000000000040da000000fe00e1
:1005e000800078001106b100030035009101b100d0
:1005f00001003c000050a1000000060080007800cf
:100600001104b100030035009101b10001003c006c
:100610000050a000000006000003b1000b003500f0
:100620009000b100080034008000b10007003500e0
:100630009001b100040034007000b10003003500e7
:100640009001b10001003c00100005000000050011
:100650001002b1000f003500e000b1000c003400c2
:10066000b000b1000b0035006000b100080034009c
:10067000b001b100070035005000b10004003400a3
:10068000b001b100030035003000b10001003c00b2
:1006900010000500000005006900e10004003500bd
:1006a0006d00e100030034000002b10001003200df
:1006b00000000500100005000a00fa008001780023
:1006c000e20f500028003e0080c78000e10f50007c
:1006d00008003200802320000000e0000500320006
:1006e00004232000252320004623200080017800d9
:1006f000040037000422200025222000462220008a
:1007000083222000144090000004e0000400350023
:100710008009eb00144090000074a0001042980083
:10072000154090000028a30003003a0015409000f7
:100730000024a000904298008001eb0007003700e1
:10074000154090000008a300fdff320063c0780050
:100750000000fb00000b78008301e800828f51004d
:10076000f7ff3a000800370030002000b0bf9f00bc
:10077000c3bf9f00d1bf9f00e2bf9f006a805700a8
:1007800000c0da006fb99700020078000080fa001c
:1007900000000600020ab900001bb9000200b80000
:1007a000810042008100430000000600881f78009d
:1007b000000478005001be004000be00040040006c
:1007c000858048000601490087814900009cbe00e1
:1007d0000294be000400e1000588e1000690e100fb
:1007e0000798e10002003100680044001008e800aa
:1007f0004f04780000000600f4874700889fbe0081
:100800008a9fbe008c9fbe008e1f78000205be002e
:100810000004be00d4b79f00e5b79f00f6b79f0065
:1008200087bf9f000000eb00c0b79f00b0b79f00dc
:10083000a0b79f0090b79f0080b79f000d042000d5
:10084000bfb097004fb09700000140000000e000eb
:100850000f003d004f08de0000007100c0b79f0090
:100860009e00070001003d0012002000a1000700cb
:1008700001003d0012002000a6000700b1000700a3
:10088000b60007000f004000c8ff07002200370035
:100890004f08de0000067100ccb79f008f000700f4
:1008a00001003d00120020009200070001003d0001
:1008b0001200200097000700a20007000fb2970067
:1008c0009fb297002fb39700bfb39700a90007000e
:1008d0000000520081805a0002015b0083815b00ae
:1008e00080b79f0091b79f00a2b79f00b3b79f004a
:1008f0000007eb009f0007000020e10001a8e100d5
:1009000002b0e10003b8e100010031001e00200048
:100910000e005600c0b79f004fb297000400e000e1
:100920000700350010002000010020006011b80011
:1009300008047000898470000a0571008b857100bd
:100940008d06e900beff3a000400e00003003d0010
:10095000820007000f00400094ff07004fa8970097
:100960000000e00004003a000fb497009fb4970025
:100970002fb59700bfb59700940007004f07780088
:100980004f06be004f05be004f04be004f01b10030
:1009900000000600881f780018002000881f7800db
:1009a00095ff07008f87e9004f04780000000600dc
:1009b000801feb0090ff07008f87e9000000060012
:1009c000889fbe008a9fbe008c1f78006e000700c3
:1009d00007003d0073000700e00f5b00e08f5b0045
:1009e00007003d00320007000006eb00040037005e
:1009f0003400070002003d002a0007001c00200010
:100a000072000700e3ff07000203be000002be0001
:100a10000c00e00001003200220007000400be00cc
:100a20000601be004f0678004f05be004f04be0011
:100a300000000600889fbe008a9fbe008c1f7800c1
:100a40005100070005003d0056000700e00f5b0065
:100a5000e08f5b0006003d0004003700190007002e
:100a600003003d006000b8006011b80010000700ee
:100a700056000700ceff07000203be000002be00c2
:100a80000c00e00001003200060007000400be0078
:100a90000601be004f0678004f05be004f04be00a1
:100aa000000006006000b8006011b80000003700c8
:100ab00004025000858258000603590087835900bc
:100ac000000006000006eb00e00f5200e08f5a0025
:100ad000e00f5b00e08f5b0000000600018040003b
:100ae00090b79f000001eb008fb097000100e0007d
:100af000000006000200700090b79f0001804000d7
:100b000080b79f000001eb00ffa897000100e00004
:100b1000000006000200700080b79f0001804000c6
:100b20006faa9700cf20de0001007000f0af9f0099
:100b300004024200250007004f18de000002720088
:100b400000000600e4af9f000804440089844c00c4
:100b50000a054d008b854d00000006003fb297004e
:100b6000cfb297005fb39700efb3970000fe2f005e
:100b7000000006003fb09700cfb097005fb197002c
:100b8000efb19700000006000205be000004be00a1
:100b9000e00f5000e08f5800e00f5900e08f59003f
:100ba000000006006000b8006011b80008045000a2
:100bb000898458000a0559008b8559001c002000c3
:100bc000e00f5200e08f5a00000006000800be004f
:100bd0000a01be00000006002800fa00889fbe003f
:100be0008a9fbe008c9fbe0003866b000c0207002c
:100bf0000028a30064003a000128a30067003a001f
:100c00000008a30062003a000108a30065003a0052
:100c10001e009000be08900081064000ed3fb1002c
:100c2000f4805700ee019000111ab8008e09900070
:100c3000311bb8009e099000311cb800511db8004e
:100c4000f485570046000700fe0190003a000700b7
:100c50008b85e8003e0007008e09900040000700e9
:100c6000ee019000340007008b85e8003800070093
:100c70008e099000400007009e0990001b18b800e4
:100c8000890440000a854800fe01900034000700f6
:100c90008b85e80038000700ee0190003000070067
:100ca0008e0990001b18b800890440000a8548008e
:100cb0000a98a30008003a000402420085824a0014
:100cc00006034b0087834b0008044c0089844c00ca
:100cd0000a054d008d06e9008482720085027300ca
:100ce0004c3add0085027200010032001500200040
:100cf000443ade001400b2004538de00cb45dd008a
:100d00000b007000c540de00cb4ddd008b80700015
:100d10004549de00cb55dd000b017100c551de00f9
:100d20000d037800d701070003f0a1000cf0a70025
:100d300003f0a000ce0137001b18b8008502400068
:100d400006834800e0834b0060044c000700370036
:100d50001b18b8000603400087834800faff3700dd
:100d60001b18b8008703400008844800e0844c004a
:100d700060054d00000006001b18b8000804400084
:100d800089844800faff37000108a300b5013a0042
:100d90005800be005801be00e3ff37000008a30062
:100da000b0013a0009047800f9ff370081037800a8
:100db000e00107000001be006000b8000478a30055
:100dc00013003a006220e10015003e000d003900da
:100dd0008301d1000281d3008180d3008301d1003f
:100de0000281d3008180d3008301d1000281d3002e
:100df0008180d3000538b000c42add00f300b200c2
:100e00008381720007f0a70003f0a0000000060035
:100e1000f3ff2700f2ff2f006110b900fbff37003e
:100e200003ff2700f7ff37008f1fd100d60107000f
:100e30008f87e9000000e00000000600801feb0043
:100e4000d10107008f87e9000000e00000000600e4
:100e50001400fa00889fbe008a9fbe008c9fbe00cf
:100e60000005be000206be00680047000c90be00f0
:100e70000a90be00ed0107006400e1001a00320094
:100e800016003e006100e1001a0032006e0490007e
:100e9000fe0490000e0b90009e0b90006011b800b5
:100ea0009e0590000b38b100d501200082817100b1
:100eb000610164008703d1000683d3008984d300d5
:100ec0000884d3008502e900f8ff3a00fe0107001c
:100ed0000df0a70001f0a00065013700f1ff270029
:100ee000f0ff2f006201370001f82700000020000a
:100ef000f7ff37006000b800f5ff37001802070061
:100f00000509780000000600809feb009e010700a5
:100f10008f87e9000000e000000006002800fa00ca
:100f2000889fbe008a9fbe008c9fbe000706780087
:100f3000878669000c003b00030478008704780072
:100f400008f0a10009f0a100840f5000858f58001f
:100f5000860f5900890f5c00030033000cf0a200db
:100f600001003a000cf0a1002d0107006400e1002f
:100f70005f003200780147006408e1006100320040
:100f80006c014700748557003200be001201be009c
:100f90003a04be001a05be001e039000be0a90006f
:100fa0008503530006003d000004fd008104fd00a0
:100fb0000205fd008305fd008703ea0005037800b4
:100fc0000df8a3000400320060041400e0841c004b
:100fd00060051d00e0851d006022b8007d03200033
:100fe0000d38e1008006eb000b0039004433dd00d2
:100ff000f300b2008301730039003700848272006d
:101000000d027800e10664008b85d1000a85d300cb
:101010008984d3000884d3008703e900f7ff3b00ed
:1010200008004000898048000a0149008b8149007e
:1010300004003b0060001000e0801800600119000f
:10104000e08119000358a300090032008d8272006c
:1010500084827200610260008301d1000281d300aa
:101060008180d3000080d3000603e8001b00370016
:101070000348a30017003a000600e0001700340000
:101080000603e9000d00a30000004800818048002d
:1010900002014900838149000348a3000f003a0080
:1010a0000600e000090034000603e90000004000eb
:1010b00081804800020149008381490001003a0013
:1010c0000003eb000348a300f5ff32006022b800e4
:1010d000020037008482720061826600e900070026
:1010e00003f0a1000cf0a70003f0a000e00037001f
:1010f000640147006408e10002003a000df8a30013
:10110000d8003a003200be001201be00d8003700fd
:101110001400fa00889fbe008a9fbe008c9fbe000c
:101120000004be000205be00680047000a90be0031
:101130000890be003d0107000070a7000bf0a10061
:101140000bf8a30020003a009e0990000e099000c1
:10115000fe0090006e0090009e029000344320003c
:1011600084825200c20032000a003c00b4fc2f000e
:101170000428e100140034008301d1000281d3006f
:101180008180d3000080d3008502e800faff3a0096
:10119000b7003700b40020000428e10007003c003d
:1011a000000040008180480002014900838149001d
:1011b0008502e900faff3a00ad003700030028007d
:1011c00002002000010037006011b8006000b80084
:1011d000a70037002800fa00889fbe008a9fbe0043
:1011e0008c9fbe0003866b008d0007006400e10049
:1011f000440032006408e1004a0032006100e1006e
:10120000460032006108e10049003200ec06470068
:101210006000b8003d02be003d03be00f4865700ea
:101220006011b8003d04be003d05be007d032000f6
:101230000b0037000000a0008d06e900130032000b
:101240000402420085824a0006034b0087834b005c
:10125000000040008180480002014900838149006c
:101260000802520089825a000a035b008b835b00ec
:10127000f0ff3b000802420089824a000a034b004b
:101280008b834b008d06e900edff3a0084827200eb
:1012900086827200f707b200878272000100320076
:1012a000150020001e0490003e0b90000603540021
:1012b000e63fb0000368a300070032000000a7006b
:1012c0000500a0008301d1000281d3008180d300fa
:1012d0000080d3000603e8008301d1000281d3001f
:1012e0008180d3000080d3000002eb000482d20092
:1012f0006400070003f0a1000cf0a70003f0a000b9
:101300005b003700640247006408e10055003200ca
:101310003400be003401be00f6ff37006108e10072
:10132000500032006011b8006000b800f1ff3700d3
:1013300003ff270002002000fbff3700889fbe004c
:10134000830478000300e0002c00350003003c001b
:101350000082700004027100260032003643200033
:10136000c50020008383cf000a0039000541b10089
:101370008283cf00070039000541b1008183cf008f
:10138000040039000541b1008083cf00010039001d
:101390000541b10085c353006022b800120032003d
:1013a0000a003b0084827200610260008301d10068
:1013b0000281d3008180d3000080d3000603e800bf
:1013c0008743e800f7ff3a000700370000004000bd
:1013d0008180480002014900838149000603e90039
:1013e0008743e900f9ff3a002600070009f0a7004b
:1013f00003f0a0004f04be000000060060001000d3
:10140000e080180060011900e0811900d3ff3b0063
:10141000033e2c00f7ff370007f0a200bffe3700a5
:10142000680447000294be000094be00fc0447001c
:101430008694be008494be00090078007b000700fb
:10144000080078007900070099007800814f70004b
:101450000b003b000800be00ce0007004f00b100ab
:1014600003003700f3ff2700f2ff2f006110b900df
:101470004f06be004f05be004f04be000080fa00bc
:101480000000060018002000570020000804530048
:101490000d003d000600200097fc2f000740e100f2
:1014a0001e00340084827200610260008301d1005a
:1014b0000281d3008180d3000080d3000804e800bb
:1014c000f8ff3a0047002000610460000504740042
:1014d000040464000d00320061004000e080480018
:1014e00060014900e081490003b8a500070032000f
:1014f0000603e8006538e10004003a008301d100ea
:101500000281d3008180d3000080d300f87f2000c7
:101510000830e10003003500080378006000b800df
:101520006011b8004433dd00f300b20083017300a2
:1015300000000600c70ade00f107b200f50fb20096
:1015400008003200e1cf4200020032000170a0002a
:1015500024000500810f700001003200040805001e
:1015600044000500810f700002003a0014000500dd
:101570008502e9000000400081c04800fcff3b00fc
:101580000170a00024000500889fbe008a9fbe0055
:101590008c9fbe000404be000605be00809fbe00f6
:1015a000829fbe0089000700040678000800be0084
:1015b0000a01be0085000700840678004f03be00c4
:1015c0004f02be008d4f76007fb0970013003300ae
:1015d000f0ff2f008b8f6b0006003b000d066600ae
:1015e0000c00a7000a00370007f0a600100020003a
:1015f0000a003700880f5200898f5a008a0f5b005b
:101600008b8f5b00030039001000200001003e00ba
:101610000000200007f0a7000000ea004f06be000f
:101620004f05be004f04be00000006008000780099
:101630005002be005003be004439de00f700b20085
:10164000f37f200003016100090032000218e1006d
:1016500016003a00850172008301730083817300d4
:101660000008200015003a00400020001300370059
:1016700085017200830173008381730005003a00c5
:1016800004a8be0006a8be00100020000b00370012
:101690000201e9000402420085824a0006034b0071
:1016a00087834b000748a300f9ff32000740a000e2
:1016b00004a8be0006a8be002000200080009800fc
:1016c0009200980000000600810020006180550013
:1016d0000b003d000b00200061fe2f000100e10027
:1016e0001d00340082817100610164008904d10011
:1016f0000884d3000000e800faff3a0071002000df
:101700006100640003007000020060000900320004
:1017100061044400e0844c000988a5000500320003
:101720008b05e8006808e10002003a008904d10056
:101730000884d300f20f20000258e10005003d00ac
:10174000c75ddd00f907b2008980750008007800e8
:10175000000006000bf827008b0078000000050051
:101760000003be0073ff07006220e10002003200a8
:101770000600be0005000500e507b100f107b20054
:1017800004f023008480700007f0a70001f0a0009f
:1017900024000500e48240001078a3000700320016
:1017a000640240001178a3003400be001401be00a2
:1017b000040032000330a700000006003500be0020
:1017c0001501be000330a0000000060005ff270041
:1017d00005826100070032000428e10001003200a8
:1017e000240005000600070001003a00440005003f
:1017f0000408050002000700f9ff3a001400050084
:101800006f826100810270008502710085027200a2
:10181000000006000001780000c2b300010037009c
:101820000201e8009240780080cf5000fcff3200b7
:10183000e9cf5000faff3200d0c2b30080cf500091
:1018400003003a000201e80014c0b30005003700ad
:101850000042eb00b0c2b30080cf500001003a005c
:101860000201e8008000eb0005fd2f0004003700b6
:101870006a08b90000804100850040000201e800cc
:101880009201fb0005804100e90f5000f8ff36008f
:101890000404e000010032008100ea000100780049
:1018a00000000600889fbe000004be000000e000ab
:1018b00003003a0078c780000800e00013003200ff
:1018c0000800be007a000700000444001804e0008d
:1018d00004003a000000eb0070c7880000047800a4
:1018e0000a0037000800be00840007000000440022
:1018f00070c788001004e000020032000058eb00be
:10190000010037000000eb0070c788000800780075
:101910004f04be0000000600800078003004e000a4
:10192000feff3a00010050000000e9000000060040
:101930000c00fa00889fbe0000047800cfb097002a
:10194000f0ff2700d0bf9f008004eb0099bf9f00ed
:1019500088bf9f00a8bf9f00200c2000b0bf9f0041
:101960007881570070805700ce0007000fb89700ad
:10197000094878000fb89700080450000800780064
:101980004f04be000080fa0000000600889fbe00e1
:101990008a9fbe008000780000c2b30001003700bb
:1019a000890078008104780039447800804f540021
:1019b000fbff3200e94f5400f9ff3200d0c2b30000
:1019c000804f540004003a00194478008184e800f4
:1019d0001ac0b300060037000045eb00b0c2b300e8
:1019e000804f540002003a00194478008184e800d6
:1019f0006022b8000a003700a20020000300200087
:101a00000400be0063fb07000b4144000281fb00a1
:101a1000030020000002410081824900394478001f
:101a20000880fb000bfd2f000b004000e90f500069
:101a3000f1ff36000a04e0000200320060021200ea
:101a4000e0821a000400be004f05be004f04be0035
:101a50000000060010417800b141510003003a0037
:101a60000000e8000204e000faff3a000300fb0077
:101a7000000006008001eb00020037008171780051
:101a80008301e800828f5100fcff3a00000006004d
:101a9000800178000001780031407800005978001a
:101aa0000004e000fcff3a0003007800000006009c
:101ab000889fbe008a1f78000005780081047800a6
:101ac0000004eb00010037000804e80068407d00d6
:101ad0000004e000050032008000fb0009007800ef
:101ae000b50507000000e000f7ff3a0008007800a5
:101af0004f0578004f04be0000000600889fbe001e
:101b00008a1f780000057800810478000004eb004b
:101b1000010037000804e80068407d000004e00090
:101b2000050032008000fb0009007800a2050700d4
:101b30000000e000f7ff3200080078004f05780051
:101b40004f04be0000000600889fbe008a1f780078
:101b5000804078000004e00021003d008040ea0061
:101b6000d0c6b30080cf5000090034008104fb00d0
:101b700042062000110009008204d800000178000c
:101b8000010078004311dd008a6921001f00370041
:101b90000100fb008369210039003700a20020000a
:101ba000110009000200d80000017800010078004f
:101bb0004311dd00030141004300dd00030040004c
:101bc0003002be002003be0042209000d2209000d0
:101bd000f221900062219000fffb07002e003700e9
:101be000d0c6b30080cf5000230034008104fb0036
:101bf00042062000110009008204d800000178008c
:101c0000010078004311dd008a7421000a014100bf
:101c1000a8002000110009000800d8004300dd00e2
:101c20000a00400040229000d022900060239000e3
:101c3000f02390000288900092889000b289900072
:101c400022899000e4fb0700801f780001027800e1
:101c5000110009008804d8000102fd004f0078003f
:101c60000402fb004322dd000a0242005403be00ce
:101c70004402be00d8ff37000100fb00837421003e
:101c8000eacf5000c5ff3c004300dd0003004000e8
:101c90005001be004000be004f0578004f04be005a
:101ca000000006008f03b000889fbe008a9fbe0020
:101cb0008c9fbe008e1f7800e0b79f00f1b79f0099
:101cc00082bf9f000000eb00a0b79f00e604370032
:101cd0008001eb0050c2b30080cf500009003200f9
:101ce0000100fb00efb09700ec040700e10f40009b
:101cf000dd043200afb097008100e800a1b79f007b
:101d0000d90437007fb1970092407800d0c2b30069
:101d100080cf50000c00320007003c006d405000a6
:101d200080cf50000d0032006b40400080cf50004b
:101d300019003a000e00370000c3b30080cf5000f6
:101d400015003a000f0037000330a0007fb2970063
:101d50000402e800f4b79f00eaff37000300a00088
:101d6000ffb297008502e800f5b79f00e5ff370056
:101d70000310a0007fb697000c06e800fcb79f0098
:101d8000e0ff37000320a0007fb097000000e800cc
:101d9000f0b79f00dbff37000318a30001003200fb
:101da0000300a1000338a300010032000320a100ba
:101db0000100fb0002fd2f0002004000e90f50006f
:101dc00010003e008000eb00c1b79f0002027800c7
:101dd0004fb197006a10b900ffb297001501fb00e0
:101de0000001410004014100c2b79f005500fb0003
:101df000f5b79f0004004000e90f50000d003e00c1
:101e0000f3ff37000006eb00ccb79f00a0c2b30081
:101e100080cf500007003a000fb89700c00078004c
:101e200080bf9f00c1b79f007fb197000201e8000b
:101e3000f2b79f00e0c2b3007fb29700944f10004a
:101e400021003a00830678000de0a0008400e8003d
:101e500064405000914f100004003200f1b79f0021
:101e60008002eb00b5b79f00100037000fbe97004f
:101e70004c0078008cbf9f00b0b79f00ffb0970068
:101e80008180e800f1b79f00130037003fb2970050
:101e90006a20b9000000410003004000b0b79f0075
:101ea000ffb297008502e800f5b79f007fb6970064
:101eb0001c01fb0003fd2f0003004100e90f50004f
:101ec000f2ff360004003700830678000dc0a00042
:101ed0000000eb00b0b79f007fb19700b2407800e0
:101ee000f2b79f00c17f9f00c0c6b30080cf5000f3
:101ef0002700320014003c006840500080cf5000a2
:101f00009d00320009003c006c40500080cf500022
:101f1000290032006b40400080cf50007200320038
:101f20000104e000560432008e00370060c6b300a2
:101f300080cf50001c0032006340400080cf500032
:101f400088003a008c00370030c7b30080cf5000c3
:101f50001c00320007003c006440500080cf50005d
:101f6000130032000040e80080cf50007d003a00ae
:101f70001100370050c7b30080cf50007d00320001
:101f80006340400080cf500076003a000b003700dd
:101f9000000028000d48a30001003a0000012000c5
:101fa00080867600ccff37000da0a00072003700bd
:101fb0000d60a000700037000d50a0000d70a00053
:101fc0006d0037008fb997004300780083bf9f00f2
:101fd000000478000000e00001003a008889210038
:101fe0008004eb00010037008104e80089007800dc
:101ff000088044001004e000fbff3a003fb2970065
:102000000400e00003003200890f5200010031009b
:10201000840478000007eb00cfb29700898f52004c
:1020200001003600098752004368de00e1066000c7
:1020300019003a000d06780009003700efb097004c
:102040000002200015040700e10f400003003200e9
:102050002fb097000000e800a0b79f000c06e80032
:102060008e0f5600f5ff3a000087eb000a0037009c
:10207000880078003100fb0001047800efb0970081
:1020800006040700e10f400003003200afb09700e4
:102090008100e800a1b79f000900e90080047800f2
:1020a000e10f4000f2ff3a000006eb000d00e000f7
:1020b0000a003a00ec033700efb09700000220005e
:1020c000f6030700e10f4000030032002fb1970034
:1020d0000201e800a2b79f000c06e8008e0f560030
:1020e000f5ff3a00e00337008fb99700430078000e
:1020f00083bf9f00cf80de0001017800820178005d
:102100000205be000004be000203be000002be00c5
:102110004822de00482edd0004027600c47f9f00c6
:102120000d48a3000a0032000404e0000800320059
:10213000e14f420006003200d1fb2f000180470032
:102140000448780018409800290020000200370059
:10215000d07f9f0019002000d2fb2f00028447008f
:10216000a6ff3700c3fb2f0003844700190020009f
:10217000a2ff37000d0cb300007020000082660043
:10218000270232000dc8a3000200320064002000c4
:10219000b4b79f000d48a300050032000fba9700a6
:1021a0004401be004400be0084bf9f00040037000d
:1021b0008fba97004500be0085bf9f00fbfa07005d
:1021c000e0af9f00f1af9f0082b79f0093b79f00e1
:1021d0006022b8006033b8006fa89700ffa897008e
:1021e0000fb197009fb197000ffb07000000e000c0
:1021f0000a003d006fa89700ffa897000fb1970055
:102200009fb1970003f0a200e0af9f00f1af9f00e5
:1022100082b79f0093b79f003d00b3000000eb0022
:1022200080a79f006022b8006033b8006fa89700b5
:10223000ffa897000fb197009fb19700fffa070022
:102240000000e000340032006fa89700ffa897005c
:102250000fb197009fb19700fdfa070003fc2f0014
:102260000381470025fb07000fa097000000e9004d
:102270006300b900a2002000110009000200d8008c
:102280008000fd0081a79f000100e00002003d00ea
:102290000100e90080a79f000fa497000840ea0012
:1022a00029fe07006faa9700ffaa97000fb39700b7
:1022b0009fb3970048fa0700a0af9f00b1af9f00ff
:1022c000c2af9f00d3af9f006022b800060020007d
:1022d00007ff2300d4fa07000000e00002003d00e1
:1022e0000800e9000b0037006022b800060020005b
:1022f000470224002fa89700bfa897004fa9970076
:10230000dfa9970000fb07000000e0000200350095
:102310000800e80080a79f003fb29700f80f520026
:1023200057003c00d0c6b300804f52002900360051
:102330000485fb0042062000110009000285d80038
:1023400000017800010478004311dd008b69210051
:102350000b0141006022b8000600200007fe2300a8
:102360000288900092889000b289900022899000a3
:1023700019fa0700a9002000809fbe001100090083
:102380000984d800000478004f00be004344dd00fb
:102390000b04440048229000d8229000682390004b
:1023a000f82390000cfa0700801f780001027800e3
:1023b000110009000985d8000102fd004f007800d6
:1023c0004322dd000b0242005403be004402be0063
:1023d0001f0037000480fb0089692100ea4f52008a
:1023e00014003600a2002000110009000280d8006d
:1023f00000017800010478004311dd00090141006b
:102400006022b8000600200007fe23004220900052
:10241000d2209000f221900062219000eef9070096
:102420004344dd00090444003802be002803be0016
:10243000070037004300dd00090040006022b800bb
:102440000600200007fe23005001be004000be0031
:10245000e1f907000002be000203be006fa897006a
:10246000ffa897000fb197009fb19700abfa070044
:10247000e0af9f00f1af9f0082b79f0093b79f002e
:102480000fa49700e90f540015003c006022b8002b
:102490006033b8006fa89700ffa897000fb19700ae
:1024a0009fb1970065fa07000000e000320032009b
:1024b0006fa89700ffa897000fb197009fb19700f2
:1024c00013fb0700e00f5000e08f5800e00f5900a9
:1024d000e08f590028003a00e10f54002600340034
:1024e0000400200005002e00b6e0220017012400a1
:1024f0002fa89700bfa897004fa99700dfa99700c2
:1025000049fa07000000e00002003d00730054009b
:10251000010037007200540080a79f000fc0970091
:1025200089fd0700a0af9f00b1af9f00c2af9f0021
:10253000d3af9f000002be000203be006fa8970049
:10254000ffa897000fb197009fb1970021fb0700ec
:10255000effa07000205be000004be006000b800ec
:102560006011b800a0a79f00b1a79f00c2a79f005d
:10257000d3a79f002e0037006fa89700ffa89700f1
:102580000fb197009fb19700e1fa07000205be0066
:102590000004be00e00f5000e08f5800e00f59002b
:1025a000e08f59000200350064fb0700130037007c
:1025b00010002000010020006011b8000800600039
:1025c000898060000a0161008b8161008b03d1006a
:1025d0000a83d3008982d3000882d30000007200ee
:1025e00081807200020173008381730053fb070036
:1025f0000002be000203be0048fa07000002be004f
:102600000203be006fa89700ffa897000fb19700c4
:102610009fb1970080fb0700a0a79f00b1a79f0074
:10262000c2a79f00d3a79f000000eb0080a79f00d8
:1026300014c0b300857f21000b0037000400fb00ad
:102640004300dd00050040005001be004000be0018
:102650000040e10001c8e10002d0e10003d8e10040
:10266000030039000442e800f44f5200f3ff3a003f
:10267000c47f9f000400fb00bfb0970000804000b3
:102680008fa09700010040004fb197000007510054
:10269000bfb197000300e000010032000e07e9001f
:1026a00063806600010032000e07e9000d28a300d8
:1026b00026003200e18066000d18a3000c003200f5
:1026c000d00220000100e00001003a000080e90093
:1026d000efb0970071020700e10f400018003200d0
:1026e0002fb297000402e800a4b79f00140037003f
:1026f0000100e00012003200efb09700000220005d
:1027000066020700e10f40000d003200afb29700f3
:102710008502e800a5b79f0009003700efb09700d9
:10272000000320005d020700e10f400003003200bb
:102730002fb697000c06e800acb79f000e07e90023
:102740000e00e000f5ff3c003d0037000d38a3000f
:102750000a0032000b003700efb0970000022000a3
:102760004e020700e10f4000030032002fb0970037
:102770000000e800a0b79f000e07e9000e00e0008f
:10278000f5ff3c00e18066000d18a3000c0032004c
:10279000d00220000100e00001003a000080e900c2
:1027a000efb097003d020700e10f40002400320027
:1027b000afb097008100e800a1b79f00200037006c
:1027c0000100e0001e003200efb097000002200080
:1027d00032020700e10f4000190032002fb19700cc
:1027e0000201e800a2b79f00150037000000fb00bf
:1027f0004300dd00817f2100010040003002be0067
:102800002003be000800be000a01be0061f80700f8
:10281000a4002000050020006033b80064f8070021
:102820000003b000efb097001c020700e10f40006a
:1028300003003200afb197008301e800a3b79f0007
:102840004f7a97000440e900c07f9f00e14f4000ad
:10285000e6ff3a000b003700efb0970000032000be
:102860000e020700e10f400003003200afb29700f4
:102870008502e800a5b79f000fa097000000e900bf
:1028800080a79f000fa097000000e000f2ff3c002f
:102890003fb6970020c1b300f20f560001003c0084
:1028a0006fe09700c07f9f00cf7897000100fb008a
:1028b0003fb1970000005100e0a79f000104e00035
:1028c00008003200efb09700e0022000f30107009b
:1028d000e10f400003003200afb197008301e80030
:1028e000a3b79f004f78970097fc07000002be0037
:1028f0000203be002fa09700bfa097004fa1970032
:10290000dfa19700b4f8070001fa07001e003700a6
:102910000000fb004300dd008c7f21000c00400024
:102920003002be002003be000800be000a01be0047
:1029300018f80700a4002000050020006033b8004c
:102940001bf807000003b000efb09700d3010700a9
:10295000e10f4000030032002fb297000402e800ac
:10296000a4b79f00cf7a97000500fb004300dd006d
:102970000c0040003002be002003be000800be0074
:102980000a01be000af807000205be000004be00ee
:102990004f7e97000c40e900c07f9f00e14f400050
:1029a000dbff3a000006eb0009003700efb09700ac
:1029b00000032000b9010700e10f400003003200ce
:1029c0002fb097000000e800a0b79f000c06e800b9
:1029d000efa09700810f5600f4ff3a000d38a300d6
:1029e000a10132000e00e0009f0134000006eb0060
:1029f000efb0970000022000a8010700e10f40009f
:102a0000030032002fb197000201e800a2b79f0037
:102a10000c06e8008e0f560093013200f4ff3700d9
:102a20000d007800000cb20028003a000d00e00014
:102a300005003d008fb997004305be004304be006a
:102a400083bf9f00140037000d48a3000b00320025
:102a50000fba97004400be0084bf9f004f89de007c
:102a6000cf91de000002be000203780082037800ee
:102a70000605be000404be00070037008fba9700a9
:102a80004500780085bf9f0000047800cfc4de00b9
:102a9000090578008a057800e00f5400e08f5c009b
:102aa000e00f5d00e08f5d0020003d003d00b300c1
:102ab0006000b8006011b800080450008984580014
:102ac0000a0559008b855900180037000d00e000f9
:102ad00005003d000fbe97004c05be004c04be0033
:102ae0008cbf9f00110037000d48a3000800320082
:102af0008fba97004500be0085bf9f000401780093
:102b0000840178000205be000004be000700370003
:102b10000fbe97004c0078008cbf9f000004780027
:102b2000090020000a0020000b0020003fb09700a1
:102b30000000e00007003a00e00f5400e08f5c0066
:102b4000e00f5d00e08f5d0002003a001100200000
:102b5000b1b79f000d0778000e0cb20000042000f2
:102b6000800f57002f00320003003c000e00e000f1
:102b7000070032003f00370000082000800f570098
:102b800014003200000c2000800f570039003a007a
:102b900014c0b300857f21000b0037000400fb0048
:102ba0004300dd00050040005001be004000be00b3
:102bb0000040e10001c8e10002d0e10003d8e100db
:102bc0002b0039000442e800f44f5200f3ff3a00b2
:102bd0002700370000012000010020006011b8002c
:102be00014c0b3000040e10001c8e10002d0e100e0
:102bf00003d8e1001e003900450020000000d0008d
:102c00008180d2000281d2008381d2008502e90056
:102c1000faff3a000442e800f04f5200f1ff3a0098
:102c20001300370080002000010020006011b80070
:102c300014c0b3000040e10001c8e10002d0e1008f
:102c400003d8e1000a0039003c0020000000d00059
:102c50008180d2000281d2008381d2000c06e9007b
:102c6000faff3a000442e800f54f5200f1ff3a0043
:102c7000c47f9f00cf7897000100fb003fb1970011
:102c8000820f500002003d00c27f9f000400370009
:102c9000bfb19700808f510001003d00b0b79f0089
:102ca0004fb297000400e000040032006380660029
:102cb000020032000402e900c4b79f000de8a3003f
:102cc0000b003200cfb297003fb697008c8f5200b6
:102cd00003003c000000eb00c0b79f000400370079
:102ce000cfb097003fb1970082805000c1b79f00de
:102cf000cf7997000300fb000002eb0094a79f0030
:102d0000cfb29700808f5200020034000080520042
:102d100090a79f000d28a30037003200e1806600d5
:102d20000d18a3000c003200d00220000100e000ca
:102d300001003a000080e900efb09700d7000700db
:102d4000e10f40000e0032002fb697000c06e8009d
:102d5000acb79f000a0037000100e0000800320015
:102d6000efb0970000022000cc000700e10f400008
:102d7000030032002fb097000000e800a0b79f00ca
:102d80009fa097000100e0000f0032000006eb005a
:102d9000efb0970000032000c0000700e10f4000e3
:102da000030032002fb197000201e800a2b79f0094
:102db0000c06e8009fa19700830f5600f4ff3a002d
:102dc0000002eb0094a79f00bfb29700c328dd006c
:102dd000007f21008080400091af9f004228dd00ed
:102de0006400500080af9f006328b900f0a79f00e7
:102df00063065000820037001fa697000c00e00019
:102e000011003200688066000f003a00000678006a
:102e1000efb0970000022000a0000700e10f400083
:102e2000030032002fb097000000e800a0b79f0019
:102e30000c06e8009fa09700810f5600f4ff3a00af
:102e40000001eb0092a79f00e18066000d18a3002f
:102e50000c003200d00220000100e00001003a0026
:102e60000080e900efb097008c000700e10f400000
:102e7000d5ff3200afb197008301e800a3b79f00f0
:102e8000d1ff37000100e000cfff3200efb0970024
:102e90000002200081000700e10f4000caff32005d
:102ea0002fb297000402e800a4b79f00c6ff3700c6
:102eb00000042000800f57003000320003003c0067
:102ec0000e00e000070032003d003700000820003f
:102ed000800f570011003200000c2000800f5700b7
:102ee00037003a001fa897003002be002003be0042
:102ef0000800be000a01be00a6f60700a4002000dc
:102f0000050020006033b800a9f6070004c3b30031
:102f100004424000c47f9f0029003700f58921004a
:102f2000d5b79f000d58a30002003a00008b210086
:102f3000d0b79f0014002000050020006033b800c7
:102f40008fa897008100e900050033000402d0003b
:102f50008582d2000683d2008783d200f9ff370032
:102f60000800be000a01be008af607006f0060007c
:102f70005fb1970062407800100037001400200015
:102f8000050020006033b8008c0178008301e9005f
:102f9000050033000402d0008582d2000683d200ef
:102fa0008783d200f9ff37000800be000a01be0087
:102fb00078f60700674060000043b000c07f9f00c4
:102fc0004f7a97000400fb00efb097003300070032
:102fd000e10f400003003200afb297008502e80025
:102fe000a5b79f001fa897006800500090af9f00f2
:102ff0008fa89700e480500081af9f0063065600c1
:10300000d0ff2f003fb197000090b900ffa19700bb
:103010000080410063005000800f5600a4ff3a007a
:103020000d38a300100032001fa297000400e0003a
:103030000d0034000006eb00efb097000002200006
:1030400016000700e10f400003003200afb2970006
:103050008502e800a5b79f000c06e8001fa09700b6
:10306000800f5600f4ff3a007fb19700b24078001d
:10307000f2b79f00c17f9f000104e00014fb3a00fb
:103080002fb097004f0778004f06be004f05be00d7
:103090004f04be008f03b10000000600889fbe00f1
:1030a0000001780001047800b10090000118a3002d
:1030b0003d0032000198a30003003a001800900080
:1030c0000000e00038003a000190a00031049800b0
:1030d00082047800f90fb200180090000000e000b0
:1030e00002003a0028009000000c7800ea8f54009b
:1030f00006003a00380090000078a30003003a0070
:1031000088007800d0002000e4ff070098009000bd
:1031100058009000808f50000b0032000100e80042
:10312000100498001800780009587800000c780006
:1031300011c0b300c08e210001487800ea8f54000e
:103140000600320019003700880078000940780036
:103150002100070080047800140037003800900038
:103160000088a3001100320018019000a800900010
:103170004800900050f5070098009000810f500023
:1031800004003200380090000003b30030049800bf
:103190008084eb000000eb001004980028009000f1
:1031a000000c7800010037008084eb0009007800f3
:1031b0004f04be000000060010417800814f51000e
:1031c000040032000000e8000204e000faff3a00c8
:1031d0000000eb00000006000200fa00889fbe001d
:1031e000a0ff9f0001047800b100900081047800e6
:1031f0000904b200020032000000fb003600370074
:103200000118a30005003a000103b300310498003f
:10321000190498000080eb002f0037005800900040
:103220000000e00006003a00480090001200200074
:10323000e680570020f507001904980024003700a5
:10324000280090000000e00008003a00808e210075
:1032500020049800000c7800200020005004980002
:10326000100498000130a00031049800180190006b
:10327000a8009000480090000ff50700280090007b
:10328000000c78000080eb00100498001800780013
:10329000aff8970001587800000c78002ff89700dd
:1032a000ea4f50000a003a00380090000088a3005e
:1032b0000700320018019000a8009000480090001c
:1032c000fdf4070019049800a8009000010c780094
:1032d000aff897000100fb004f04be000080fa0029
:0432e00000000600e4
:020000040000fa
:020000040005f5
:0457f400021e000091
:020000040000fa
:020000040005f5
:0457f800bdfa0000f6
:020000040000fa
:020000040005f5
:0457fc007f3e0000ec
:020000040000fa
:10000800ec020000ec020000ec020000ec02000030
:10001800ec020000ec020000ec020000ec02000020
:10002800ec020000ec020000ec020000ec02000010
:10003800ec020000ec020000ec020000604100004d
:10004800ec020000ec020000ec0200008c3700001b
:1000580074370000ec020000ec020000ec02000023
:10006800ec020000ec020000ec020000ec020000d0
:10007800ec020000ec020000ec020000ec020000c0
:10008800ec020000ec020000ec020000ec020000b0
:10009800ec020000ec020000e2370000ca37000062
:1000a800ec020000ec020000ec020000ec02000090
:1000b800ec020000ec020000ec020000ec02000080
:1000c800ec020000ec020000ec020000ec02000070
:1000d800ec020000ec020000ec020000ec02000060
:1000e800ec020000ec020000ec020000ec02000050
:1000f800ec020000ec020000ec020000ec02000040
:10010800ec020000ec020000ec020000ec0200002f
:10011800ec020000ec020000ec020000ec0200001f
:10012800ec020000ec020000ec020000ec0200000f
:10013800ec020000ec020000ec020000ec020000ff
:10014800ec020000ec020000ec020000ec020000ef
:10015800ec020000ec020000ec020000ec020000df
:10016800ec020000ec020000ec020000ec020000cf
:10017800ec020000ec020000ec020000ec020000bf
:10018800ec020000ec020000ec020000ec020000af
:10019800ec020000ec020000ec020000ec0200009f
:1001a800ec020000ec020000ec020000ec0200008f
:1001b800ec020000ec020000ec020000ec0200007f
:1001c800ec020000ec020000ec020000ec0200006f
:1001d800ec020000ec020000ec020000ec0200005f
:1001e800ec020000ec020000ec020000ec0200004f
:0801f800ec020000ec02000023
:020000040000fa
:10020800ec020000ec020000ec020000ec0200002e
:10021800ec020000ec020000ec020000ec0200001e
:10022800ec020000ec020000ec020000ec0200000e
:10023800ec020000ec020000ec020000604100004b
:10024800ec020000ec020000ec0200008c37000019
:1002580074370000ec020000ec020000ec02000021
:10026800ec020000ec020000ec020000ec020000ce
:10027800ec020000ec020000ec020000ec020000be
:10028800ec020000ec020000ec020000ec020000ae
:10029800ec020000ec020000e2370000ca37000060
:1002a800ec020000ec020000ec020000ec0200008e
:1002b800ec020000ec020000ec020000ec0200007e
:1002c800ec020000ec020000ec020000ec0200006e
:1002d800ec020000ec020000ec020000ec0200005e
:1002e800ec020000ec020000ec020000ec0200004e
:1002f800ec020000ec020000ec020000ec0200003e
:10030800ec020000ec020000ec020000ec0200002d
:10031800ec020000ec020000ec020000ec0200001d
:10032800ec020000ec020000ec020000ec0200000d
:10033800ec020000ec020000ec020000ec020000fd
:10034800ec020000ec020000ec020000ec020000ed
:10035800ec020000ec020000ec020000ec020000dd
:10036800ec020000ec020000ec020000ec020000cd
:10037800ec020000ec020000ec020000ec020000bd
:10038800ec020000ec020000ec020000ec020000ad
:10039800ec020000ec020000ec020000ec0200009d
:1003a800ec020000ec020000ec020000ec0200008d
:1003b800ec020000ec020000ec020000ec0200007d
:1003c800ec020000ec020000ec020000ec0200006d
:1003d800ec020000ec020000ec020000ec0200005d
:1003e800ec020000ec020000ec020000ec0200004d
:0803f800ec020000ec02000021
:020000040000fa
:1032e40053500000492000003d20000025750000d7
:1032f4000d0a0000004d0000454f0000570d00006e
:103304000a00000000530000656e000064690000bc
:103314006e6700003a20000022250000732200009e
:103324000d0a0000002000002c090000004e0000df
:103334006f200000656c0000656d0000656e000084
:10334400742000006e6100006d65000064200000c0
:1033540025730000200000007769000074680000f5
:10336400206900006e730000746100006e63000049
:10337400652000002564000020000000657800003e
:1033840069730000747300002e0d00000a00000031
:10339400554900004e540000002500007320000031
:1033a4003d200000257500000d0a000000490000c2
:1033b4004e54000000250000732000003d20000052
:1033c400256400000d0a000000430000484100008d
:1033d4005200000025730000203d0000202500005d
:1033e400630d00000a000000464c00004f4100003d
:1033f4005400000025730000203d0000202500003b
:10340400660d00000a000000456c0000656d0000b8
:10341400656e000074200000257300002069000020
:10342400732000006e6f000074200000616e0000c5
:10343400206900006e7000007574000020740000a4
:1034440079700000652e00000d0a00000050000095
:103454006c610000746600006f7200006d20000053
:10346400696e0000666f0000726d000061740000f8
:10347400696f00006e3a00000d0a000000090000a8
:10348400736900007a6500006f6600002869000017
:103494006e740000292000003d2000002564000017
:1034a4000d0a000000090000736900007a6500003d
:1034b4006f66000028630000686100007229000044
:1034c400203d000020250000640d00000a000000db
:1034d40009730000697a0000656f00006628000027
:1034e400736800006f72000074290000203d000022
:1034f40020250000640d00000a000000097300008c
:10350400697a0000656f0000662800006c6f000097
:103514006e670000292000003d20000025640000a3
:103524000d0a000000090000736900007a650000bc
:103534006f660000286600006c6f00006174000074
:10354400292000003d200000256400000d0a000031
:1035540000090000736900007a6500006f660000ce
:10356400286400006f750000626c0000652900008b
:10357400203d000020250000640d00000a0000002a
:10358400696e000070750000740000006f75000023
:103594007470000075740000006300006163000033
:1035a400686500005b250000755d0000203d00009b
:1035b40020250000752c000020250000732c00003d
:1035c400207300006c6f000074200000257500005b
:1035d4000d0a0000006300006163000068650000dc
:1035e4005b250000733a0000256400005d200000a4
:1035f4003d20000025640000202800002573000001
:103604002c200000736c00006f7400002025000063
:10361400642900000d0a00000068000061730000c6
:103624006828000025730000292000003d200000c8
:10363400256400000d0a0000006100006c6c0000ad
:103644000053000050490000204d0000454d00008b
:103654005b25000030320000755d0000203d000055
:1036640020250000750d00000a00000053500000e2
:10367400492000004d4500004d5b00002575000009
:103684005d2000003d200000257500000d0a0000ab
:103694000053000050490000204900004e4600003d
:1036a4004f5b0000257500005d2000003d200000f8
:1036b400257500000d0a000000440000617500003b
:1036c40067680000746500007263000061720000a6
:1036d400642000007479000070650000733a0000f3
:1036e4000d0a000000090000536c00006f74000014
:1036f40020250000643a000020250000732000000b
:1037040028250000642900000d0a00000054000070
:103714006573000074200000667500006e6300008d
:10372400746900006f6e000020300000310a000050
:103734000053000050490000204d0000454d00009a
:103744005b250000645d0000203d00002025000092
:10375400750d00000a00000061630000744400005d
:103764006562000075670000312000003d20000004
:10377400256900000d0a0000007600006172000057
:103784004164000064720000203d00002025000018
:10379400640d00000a6f000075740000203d0000f5
:1037a40020250000640d00000a0000006163000091
:1037b400744300006c7200005374000075620000d2
:1037c400436d000064280000292000003d20000013
:1037d400256400000d0a000000450000727200001c
:1037e4006f7200003a200000436100007264000020
:1037f400202500007320000025640000206e0000d6
:103804006f740000206600006f7500006e64000095
:103814000d0a0000000000004745000054000000ad
:103824005345000054000000434c00004541000093
:10383400527c0000434c000052000000524500003e
:103844004144000000570000524900005445000064
:10385400004900004e54000045520000564100004b
:103864004c00000053500000490000005245000085
:103874005345000054000000484500004c4c000033
:103884004f2000004b490000545400005900000030
:10389400534c00004f5400002052000045530000d8
:1038a400434100004e000000534500004e44000018
:1038b400005000004c410000544600004f520000ec
:1038c4004d000000445500004d500000204300000e
:1038d40041430000484500000048000041530000f7
:1038e40048000000000000000e9c0000541e000070
:1038f400129c0000641e0000169c0000741e000050
:10390400209c00002a1f0000259c00004820000085
:103914002b9c00002e210000349c0000841e00001b
:10392400389c0000b61e00003e9c0000c21e000031
:103934004a9c0000d21e0000569c0000e01e0000bd
:103944005b9c00003e210000649c0000ce2100002e
:103954006f9c000094220000749c00000000000092
:1039640053500000492000004d4500004d00000068
:10397400534c00004f54000053000000534c00000f
:103984004f540000204900004e4600004f00000044
:10399400434100005244000000540000455300001d
:1039a40054000000b29c0000c0220000ba9c000039
:1039b400b0230000c09c0000f4230000ca9c000057
:1039c4005e230000cf9c000008240000749c0000cb
:1039d400000000004445000042550000473100004b
:1039e400005300004c4f000054000000ec9c000009
:1039f40068240000f39c00008c240000ca9c000092
:103a0400a0240000749c0000000000005354000037
:103a14005542000000000000089d0000fa24000048
:103a2400749c000000000000536c00006f740000e0
:103a34002025000064200000746900006d6500000a
:103a4400642000006f750000742e00002020000028
:103a540000440000617400006120000066720000f0
:103a64006f6d0000207300006c6f00007420000074
:103a740025640000206300006f720000727500006e
:103a840070740000656400002e2000002000000017
:103a94004173000073690000676e000065640000f4
:103aa40020610000732000004f500000454e0000cc
:103ab4000d0a0000004f0000706500006e00000059
:103ac4004350000055000000506f0000776500006f
:103ad4007220000053750000707000006c790000c3
:103ae400004c0000564c00005300000048560000f3
:103af4004c530000004500006e760000697200001f
:103b04006f6e00006d6500006e74000000470000d9
:103b14004644000045540000005500006e6100005a
:103b240073730000696700006e65000064000000a4
:103b3400556e00006b6e00006f7700006e00000091
:103b4400323100003a320000343a000032330000cf
:103b5400004a0000756e000020200000382000009c
:103b64003230000031320000000d00000a4600002f
:103b74004f4300004520000043480000415300002b
:103b8400534900005320000043500000552000001a
:103b9400424f0000415200004420000042750000e2
:103ba400696c0000742000006f6e00002025000086
:103bb400732000006174000020250000730d0000d4
:103bc4000a000000200900000045000052520000d5
:103bd4002025000030340000640d00000a000000bd
:103be40052440000590d00000a0000004361000027
:103bf400726400002054000079700000653a0000ef
:103c040020250000640d00000a000000436100004c
:103c140072640000204e0000616d0000653a0000ef
:103c240020250000730d00000a000000566100000a
:103c340072690000616200006c650000204e0000a3
:103c4400616d0000657300003a0d00000a00000079
:103c5400286900006e70000075740000290d0000d2
:103c64000a000000286f00007574000070750000e1
:103c7400742900000d0a0000003f00000d0a000036
:103c840000000000200900000020000000300000b7
:103c9400313200003334000035360000373800007c
:043ca40039000000e3
:020000040000fa
:103ca8000200fa00000f78005200200041cd2900e0
:103cb8001e007800b20d07000080fa000000060020
:103cc8000200fa00000f78005200200081cf29007e
:103cd8001e007800aa0d07000080fa000000060008
:103ce8000200fa00000f780052002000e1d02900fd
:103cf8001e007800a20d07000080fa0000000600f0
:103d08000600fa00200798002e009000bff6070072
:103d1800000f780010002000db0f07001e0078005d
:103d2800c60f0700100798000000eb00d60f070029
:103d38001e009000801f780020972900801f7800bf
:103d4800804b2100f8f60700e4875700814b2100db
:103d5800200020009a0b07000000eb000080fa000a
:103d6800000006000200fa00000f78000000fe00c4
:103d78000000eb000080fa00000006000200fa00d4
:103d8800000f7800d1972900200020008c0b070035
:103d98000000eb000080fa00000006000200fa00b4
:103da800000f7800fd110700610407000000eb0018
:103db8000080fa00000006000600fa0010079800cc
:103dc8001e009000410307000000e00003003200dd
:103dd800100020002007980019003700419829009a
:103de8000000eb00adf60700000f78001e00780019
:103df800801f780050982900801f7800804b210090
:103e0800c9f60700e4875700814b210020002000f5
:103e18006b0b0700100020009b0f07001e007800a6
:103e2800bbf60700800078001e007800a00f07008e
:103e38000000eb00940f07000000eb00200798003b
:103e48002e0090000080fa00000006001600fa001c
:103e5800100f98005099290040079800ce00900054
:103e68001e0890008df6070030079800ce009000dd
:103e78000000eb0089f6070064f6070020079800a9
:103e8800ce0090000000eb0084f6070010079800b1
:103e98003e009000e70207003e0090009cf60700f5
:103ea800800078003e009000701207008040780083
:103eb8002e00900000cf40006000b8007007980006
:103ec800010f98006d0047006c014700ea004700a9
:103ed800800178001e407800621107004e4890006b
:103ee800ef4f50001d003a003e009000801f780000
:103ef80090992900801f7800804b21008af60700de
:103f0800e4875700814b2100200020002c0b07007c
:103f18002e0090000000e0000a0032002e01900000
:103f2800821f7800e09a2900801f7800804b2100ca
:103f38007df60700e4875700814b21002000200010
:103f48001f0b0700019c2900200020001c0b070004
:103f580013002000230f9800480037001e0090002f
:103f68000000e00005003200a19c29001e0090001e
:103f7800570c07000000e0000a0032005e009000c5
:103f8800801f78003e009000801f7800f09c290078
:103f9800801f7800804b210063f60700e6875700f2
:103fa80031003700919d29001e009000480c070041
:103fb8000000e0000a0032005e009000801f7800d8
:103fc8003e019000821f7800d09d2900801f780054
:103fd800804b210054f60700e6875700220037007f
:103fe800719e29001e009000390c07000000e000b7
:103ff8000a0032005e009000801f7800be01900029
:10400800831f7800c09e2900801f7800804b210004
:1040180045f60700e687570013003700619f29001f
:104028001e0090002a0c07000000e0000e0032007d
:10403800ee0047006a0047001001be008288be00fb
:104048007e0090008e089000809fbe00be01900008
:10405800831f7800c09f2900801f7800804b2100b3
:1040680031f60700e8875700814b21002000200027
:10407800d30a07000000eb00200f98002e089000dc
:104088000080fa00000006002000fa00600f980087
:1040980050992900400f9800ce0890006e089000b3
:1040a800fef50700300f9800ce0890000000eb00e6
:1040b800faf50700200f9800ce0890000000eb00ea
:1040c800f6f50700d1f50700100f9800ce0890000c
:1040d8000000eb00f1f50700000f98002e08900093
:1040e800540207002e08900009f6070080007800a7
:1040f8002e089000dd110700804078001e0890000f
:1041080000c04000604f98006000b800008fbe00fb
:104118007b0047007a014700800178008000eb00af
:104128006e489000cf1007002e589000ef4f5000b7
:104138001d003a002e089000801f780090992900f1
:10414800801f7800804b2100f7f50700e4875700af
:10415800814b210020002000990a07001e089000ca
:104168000000e0000a0032001e089000801f78005e
:10417800e09a2900801f7800804b2100eaf50700ab
:10418800e4875700814b2100200020008c0a07009b
:10419800019c290020002000890a07001000200047
:1041a800700f9800280037003e589000e14f5000eb
:1041b8000d0032002e089000801f780060a02900b2
:1041c800801f7800804b2100d7f50700e48757004f
:1041d800814b210020002000790a070010002000f0
:1041e800700f9800180037003e08900087f5070008
:1041f800500798006e4890000080fb005e01900018
:10420800800040000008210000804000020878007b
:104218005e009000801f78002e089000801f7800b4
:10422800d09d2900801f7800804b2100bef5070033
:10423800e6875700814b210020002000600a070014
:104248000000eb00700f98007e0890000080fa00d4
:10425800000006000200fa00000f78001e00780037
:104268006af50700a0b488000000eb000080fa009f
:10427800000006000200fa00000f7800804b2100c1
:1042880091a229001700090031587800814b2100bc
:10429800200020004a0a070020002000801f780024
:1042a80010a42900801f7800804b21009ef507008c
:1042b800e4875700814b210020002000400a0700b6
:1042c80010002000801f780050a52900801f78006a
:1042d800804b210094f50700e4875700814b2100ab
:1042e80020002000360a070020002000801f7800e8
:1042f800a0a62900801f7800804b21008af50700be
:10430800e4875700814b2100200020002c0a070079
:1043180040002000801f780000a82900801f780036
:10432800804b210080f50700e4875700814b21006e
:1043380020002000220a070040002000801f78008b
:1043480050a92900801f7800804b210076f50700ce
:10435800e4875700814b210020002000180a07003d
:1043680040002000801f7800b0aa2900801f780034
:10437800804b21006cf50700e4875700814b210032
:10438800200020000e0a07000000eb000080fa0061
:10439800000006001400fa00500798005e00900024
:1043a8005bf50700100798001e0090000000e00071
:1043b80031003a000000eb00200798002900370080
:1043c8002e0090000042780069004700680147000d
:1043d800e6004700800178000440780021100700bb
:1043e8000e489000e74f50001b003e000e4890001a
:1043f8000080fb00100f98001e4890000004e000a9
:104408000300320020ac2900000f9800020037009a
:1044180081ac2900010f98003e0090001e09900011
:10442800821f78008e089000811f7800801f780016
:104438002e019000821f7800f0ac2900801f7800c0
:10444800804b210038f50700ea875700814b21008f
:1044580020002000da0907002e0090000000e80084
:1044680020079800ae009000f00f2000808f5000c9
:10447800d3ff3600270037009e0090005e009000b2
:10448800fa100700004f78006900470068014700ec
:10449800e6004700800178001e407800f10f070011
:1044a8000e4890000080fb00700798001e4890009e
:1044b8000004e0000300320020ac290060079800e7
:1044c8000200370081ac2900610798003e00900087
:1044d8009e80fb007e019000821f78006e01900094
:1044e800821f7800801f7800811f78005e0090008e
:1044f800801f7800d0ae2900801f7800804b2100f3
:1045080009f50700ec875700814b210020002000a7
:10451800ab0907000000eb000080fa00000006006d
:104528000200fa00000f78001e007800f8f4070077
:10453800800078001e007800cc1007000080fb0087
:10454800801f78001e007800801f7800f0b02900d6
:10455800801f7800804b2100f3f40700e68757009e
:10456800814b210020002000950907000000eb0086
:104578000080fa00000006000600fa0020079800f4
:104588002e009000a1f4070010079800f1b129004f
:104598002e009000ce0a07000000e0001a0032004a
:1045a8000000eb00100798001300370021002000de
:1045b8001e0090001e0e0700000f78001e007800f5
:1045c800801f78001e009000801f780030b22900fc
:1045d800801f7800804b2100d3f40700e68757003e
:1045e800814b210020002000750907001e00900063
:1045f8000000e800100798001e009000ef0f500020
:10460800eaff360010003700210020001e0090004d
:10461800070e0700000f78001e007800801f780042
:104628001e009000801f780080b32900801f78004a
:10463800804b2100bcf40700e6875700814b21001e
:10464800200020005e0907000000eb000080fa004f
:10465800000006000600fa00200798002e009000cf
:104668006af4070010079800110020001e0090004f
:10467800ef0d0700000f78001e007800801f7800fb
:104688001e009000801f7800b0b42900801f7800b9
:10469800804b2100a4f40700e6875700814b2100d6
:1046a80020002000460907000000eb000080fa0007
:1046b800000006000a00fa00300798003e0090004b
:1046c800020107000000e000030032001000200093
:1046d800400798001d003700519929000000eb00a1
:1046e8006ef40700200798002e00900088f4070059
:1046f800800078002e0090005c1007000080fb000e
:10470800100798001e00900021002000c80d070027
:10471800000f78001e007800801f78002e0090009f
:10472800801f7800d09d2900801f7800804b2100d1
:104738007df40700e6875700814b21002000200008
:104748001f0907000000eb00400798004e0090008a
:104758000080fa00000006000600fa002007980012
:10476800f1b5290020002000150907000000eb0022
:10477800000f7800140037001e007800c8020700f8
:104788000080fb00100798001e009000ed02070053
:104798009e009000811f7800801f78001e0078001e
:1047a800801f780050b72900801f7800804b2100b7
:1047b8005df40700e8875700814b210020002000a6
:1047c800ff0807001e0fe800710020009e8f1000f0
:1047d800e9ff34000000eb000080fa00000006004a
:1047e8000400fa00100798001e00900007f4070064
:1047f800000f78001e007800150307000000eb008a
:104808000080fa00000006000200fa00000f78009d
:10481800804b210091b82900110009003158780017
:10482800814b210020002000e50807000000eb0074
:104838000080fa00000006000a00fa00400798000d
:1048480050992900000f78009e0078004e009000d3
:1048580012f40700100798001e00900049f40700a2
:10486800300798009e0078000000eb000bf407006a
:10487800100798001e00900042f4070020079800d7
:10488800ae0090003e0090008c0d07002e009000b6
:10489800801f78003e009000801f7800b0b9290082
:1048a800801f7800804b21001ff40700e68757001f
:1048b800814b210020002000c10807000000eb0008
:1048c8000080fa00000006000200fa00000f7800dd
:1048d8001e007800cdf3070070b4880070b4800023
:1048e800801f7800e0ba2900801f7800804b2100e3
:1048f8000df40700e4875700814b210020002000b9
:10490800af0807000000eb000080fa000000060076
:104918000400fa00100798001e009000bbf307007f
:10492800000f78001e007800b70107000000eb00b8
:104938000080fa00000006000a00fa00300798001c
:104948003e009000610007000000e0000300320014
:1049580010002000400798002100370051992900d5
:104968000000eb00cdf30700200798002e00900010
:10497800e7f30700800078002e009000bb0f0700c7
:104988000080fb0010079800519929000000eb00f7
:10499800c2f307009df30700000f78001e00900087
:1049a8009e007800450d07001e007800801f7800e3
:1049b8001e009000801f7800f0bb2900801f78003f
:1049c800804b2100d8f30700e6875700814b210070
:1049d800200020007a0807000000eb00400798003c
:1049e8004e0090000080fa00000006000400fa0063
:1049f800100798001e00900084f30700000f78004d
:104a08001e007800801f780080bd2900801f780074
:104a1800804b2100c4f30700e4875700814b210035
:104a280020002000660807000000eb000080fa0064
:104a3800000006000400fa00100798001e0090000d
:104a4800000f7800080037001e007800104078003a
:104a58000000fb00e0ee0700804078001e007800b0
:104a6800014878001e0fe8001e007800104078000a
:104a78000004e000f4ff3a000080fa00000006009d
:104a88000400fa00100798001e009000000f78003c
:104a9800080037001e007800104078000000fb0076
:104aa800d4ee0700804078001e00780001487800a6
:104ab8001e0fe8001e007800104078000004e00097
:104ac800f4ff3a000080fa00000006001200fa0025
:104ad8007007980050992900400798000080eb0063
:104ae800300798000000eb00000f7800ce0090001f
:104af8007e00900069f30700600798006e00900040
:104b0800ccff0700ce0090000000eb0063f3070025
:104b1800500798005e0090003cf3070010079800cb
:104b28000000eb0020079800110037002e009000cd
:104b3800ef010700800078006e009000c3f30700c3
:104b48000000e00007003a001e0fe8001e00900079
:104b58009e0f100003003a002e00900030079800c6
:104b6800060037002e0090000000e800200798009b
:104b78002e009000e70f5000ecff36003e0090003a
:104b8800e10f40000f003a001e009000801f7800df
:104b98006e009000801f7800f0be2900801f78000a
:104ba800804b210060f30700e6875700814b210006
:104bb800200020000208070010002000000f9800c5
:104bc800040037003e0090000f0107000000eb00d2
:104bd800000f98000e0890000080fa000000060000
:104be8000a00fa0020079800310798000000eb003f
:104bf800000f78003e0090000000e00003003a003b
:104c080020002000400798001c0037000000eb003f
:104c1800100798000800370040c2a90011002000c2
:104c28002e009000820c0700000f78001e009000f4
:104c38000000e800100798009e009000703e2000d9
:104c4800808f500002003e001e00e000f2ff32009c
:104c58003e0090001e0878009e009000703e2000e4
:104c6800808f500003003600100020004007980095
:104c7800020037000000eb00400798004e0090004b
:104c88000080fa00000006001400fa00005798009f
:104c98000e509000730107000000eb0050079800c9
:104ca8002a003700ec0047005e009000ccff0700a8
:104cb800000f78001e00e000160032000e50900031
:104cc8008080fb00801020000088b90080007800f8
:104cd8000080200000804000821020008000eb004f
:104ce80062f307000e5090008080fb0080102000c7
:104cf8000088b90080007800008020008080400093
:104d0800f0c0b300804878001e007800100f9800ab
:104d1800840037000e5090008080fb008010200037
:104d28000088b900800078005e0090008080400014
:104d380000802000808040006e009000804878004d
:104d48005e0090000000e80050079800de00900028
:104d580060102000808f5000d2ff36000e50900067
:104d68008080fb00801020000088b9008000780057
:104d7800008020000080400010407800ef4f500075
:104d8800160036000e5090008080fb008010200036
:104d98000088b90080007800008020000080400072
:104da800821020008000eb0030f307000e509000c6
:104db8008080fb00801020000088b9008000780007
:104dc8000080200080804000f0c0b3008048780058
:104dd80030002000100f9800520037000000eb0050
:104de800400798000000eb00500798003f0037008c
:104df8000e5090008080fb00801020000088b900d1
:104e0800e600400000802000008040008000e800ac
:104e18004e00900000804000300798003e0090004f
:104e2800bbf20700404798004e4090008080fb008e
:104e38003e0090008d0e0700204798004e409000dd
:104e48008080fb004e009000010040004007980061
:104e58000e5090008080fb004e0090000000e8009b
:104e6800400798004e019000801020000088b9008b
:104e780002004000e6004000108020000080400052
:104e880010407800304798004e0090000000e8007d
:104e9800400798006e0147008001eb008000eb009e
:104ea8002e4090006f0d07006e489000ef4f5000a5
:104eb800030032002e4090000040e8002047980090
:104ec8006e489000ef4f5000f2ff3a00be4190004c
:104ed8000e5190008080eb002e409000080d0700d6
:104ee8005e0090000000e800500798000e50900007
:104ef8008080fb00801020000088b900e600400098
:104f08000080200000804000104078008080fb0076
:104f18005e009000808f5000b5ff3e000000eb005f
:104f2800100f98001e0890000080fa00000006008c
:104f38000600fa000000eb00000f78000040eb00cc
:104f4800204798002b0037002e4090004eff0700a6
:104f5800000f78001e007800200798002e009000af
:104f6800e10f5000040032002e009000e30f5000c3
:104f78000d003200170037002e4090000080fb0023
:104f8800801f780060d12900801f7800000421006c
:104f980065f20700e4875700010421002000200083
:104fa800070707000b0037002e4090000080fb0029
:104fb800801f7800b0d22900801f780000042100eb
:104fc80059f20700e487570001042100200020005f
:104fd800fb0607001e00e00003003200a1d42900f0
:104fe80020002000f60607002e4090000040e80050
:104ff800204798002e409000e74f5000d2ff36001f
:105008000080fa00000006000400fa00004f780053
:105018001e80fb00100798001e009000e30f500050
:10502800410032001e009000e30f50000a003c00cf
:105038001e009000e10f5000210032001e00900079
:10504800e10f50002b003c001e0090000000e00023
:105058000e003200750037001e009000e50f50006a
:105068004b0032001e009000e50f50003b00350059
:105078001e009000e60f5000520032001e00900003
:10508800e70f50005c003200680037001100200074
:105098000000eb00c40107008000eb0010002000b6
:1050a800c10107008000eb0020002000be010700be
:1050b8008000eb0030002000bb01070067003700cc
:1050c800110020000000eb00b701070011002000cc
:1050d80010002000b40107008000eb002000200031
:1050e800b10107008000eb0030002000ae0107008e
:1050f8005a003700110020000000eb00aa01070049
:105108008000eb0010002000a7010700110020001c
:1051180020002000a40107008000eb0030002000e0
:10512800a10107004d003700110020000000eb002e
:105138009d01070011002000100020009a010700bf
:105148001100200020002000970107008000eb00dc
:1051580030002000940107004000370011002000b3
:105168000000eb00900107008000eb001000200019
:105178008d0107008000eb00200020008a01070055
:10518800110020003000200087010700330037009d
:10519800110020000000eb0083010700110020002f
:1051a80010002000800107008000eb002000200094
:1051b8007d01070011002000300020007a0107005f
:1051c80026003700110020000000eb0076010700e0
:1051d8008000eb0010002000730107001100200080
:1051e800200020007001070011002000300020007e
:1051f8006d01070019003700110020000000eb00c6
:105208006901070011002000100020006601070056
:105218001100200020002000630107001100200079
:1052280030002000600107000c0037008000eb0010
:105238000000eb005c0107008000eb00100020007c
:10524800590107008000eb002000200056010700ec
:105258008000eb0030002000530107000080fa00b6
:10526800000006000200fa00004f78001e40780097
:1052780065ff070010002000830a07000080fa007d
:10528800000006000000fa0000c0eb005eff070007
:105298000000eb007c0a07000080fa00000006000e
:1052a8000400fa00004f780070c0b3009e4f100051
:1052b8000a003e009e80fb00801020000088b90094
:1052c80080007800008020000080400010407800b6
:1052d8000080fb0010079800020037000000eb0078
:1052e800100798001e0090000080fa0000000600d9
:1052f8000600fa00204798002e409000e74f500023
:105308000b003e002e4090008080fb0080102000a3
:105318000088b900800078000080200000804000ec
:10532800000fe8001e0078002007980002003700f0
:105338000000eb00200798002e0090000080fa0083
:10534800000006000600fa00004f78001e80fb00ef
:10535800200798002e009000e50f50002e00320024
:105368002e009000e50f500011003c002e00900028
:10537800e20f50001f0032002e009000e20f500094
:1053880004003c002e009000e10f5000160032008f
:105398002a0037002e009000e30f5000180032005a
:1053a8002e009000e40f5000180032002300370050
:1053b8002e009000e90f500004003c002e009000e1
:1053c800e70f50001a003d00160037002e0090002d
:1053d800ef0f50000100320018003700d0d5290027
:1053e800100798001700370020d6290010079800ea
:1053f8001400370060d62900100798001100370004
:1054080030d72900100798000e00370080d72900f0
:10541800100798000b003700d0d729001007980014
:105428000800370090d829001007980005003700b9
:10543800f0d829001007980002003700a0d92900e9
:10544800100798001e0090000080fa000000060077
:105458000200fa00004f780070c0b3009e4f1000a1
:1054680007003e009e80fb00801020000088b900e5
:105478008000780000802000008040009a0c07001f
:105488000080fa00000006000e00fa00500798009d
:105498000000eb00100798000000eb0040079800a0
:1054a8003f0037005e009000e70040001e009000bb
:1054b8000080400016f10700300798005e00900059
:1054c800e70040001e00900000804000be009000f1
:1054d800e60c0700504798009e0090003e009000a0
:1054e80000804000100798001e0090000000e800af
:1054f800100798001e009000de0090006600400033
:105508000100400010409000404798001e009000a5
:105518000000e800100798004e4090000080fb0053
:10552800600798006e0090000000e0000400320060
:105538006e009000e10f50000d003200150037009a
:105548005e4090000080fb0021002000380a070020
:10555800000f78005e4090000080fb008000400053
:1055680000082100008040001e087800090037006c
:105578005e4090000080fb00800040000008210091
:1055880000804000900078005e4090000080fb00a2
:105598004a0a07004e0090000000e8004007980003
:1055a8005e009000604090008080fb004e009000fc
:1055b800808f5000bbff3e000080fa00000006000c
:1055c8000200fa000000eb00000f78001500370019
:1055d8009e007800801020000088b90080007800c4
:1055e800008020000080400010407800ef4f5000fd
:1055f8000b0032001e0078001aff07009e0078009a
:10560800801020000088b900800078000080200009
:10561800008040009cff070030c6b30011ff070060
:105628001e0fe800700020009e0f1000e8ff3600f3
:105638000080fa00000006000000fa00c802a90075
:10564800c822a900c862a900c882a900c902a90085
:10565800c922a900c982a900c9a2a9000000eb00bb
:10566800b0b488000000eb00b0b488000000eb0084
:10567800b0b488000000eb00b0b488000000eb0074
:10568800b0b488000000eb00b0b488000000eb0064
:10569800b0b488000000eb00b0b488000000eb0054
:1056a800b0b488000000eb00b0b488000000eb0044
:1056b800b0b488000000eb00b0b488000000eb0034
:1056c800b0b488000000eb00b0b488000000eb0024
:1056d800b0b488000000eb00b0b488000000eb0014
:1056e800b0b488000000eb00b0b488000000eb0004
:1056f800b0b488000000eb00b0b488000000eb00f4
:10570800b0b488000000eb00b0b488000000eb00e3
:10571800b0b488000000eb00b0b4880000000000be
:10572800cd82a90000000000cda2a9000000000061
:10573800cdc2a90000000000cde2a90000000000d1
:10574800e4c2a90000000000e4e2a9000000000093
:10575800cc62a90000000000cc22a90000000000d3
:10576800ec02a90000000000ec22a90000000000e3
:10577800ec42a90000000000cd02a90000000000d2
:10578800cd22a90000000000dca2a9000000000052
:10579800f522a900000000000000eb00b0b488006a
:1057a8000080fa00000006000800fa00000f7800e8
:1057b800110798001e0090000000e000020032006f
:1057c8001000200010079800000000001e0078005c
:1057d8006101b9002207980033079800f000200003
:1057e800010020002e019000be019000800f5100a2
:1057f800818f5900b2003e002e009000be0090003c
:10580800006001000f00370019003700230037003f
:105818002d003700340037003e00370045003700c0
:105828004f00370059003700620037006c0037001e
:10583800760037007f003700890037009300370073
:105848009d0037001e0090006140600061406000cc
:105858004401dd00d12c200091407800f0ceb30047
:1058680000c0600002407000cde2b700940037002d
:105878001e00900061406000614060004501dd004d
:10588800d12c200091407800f0cdb30000c060001a
:1058980002407000cde2b700890037001e0090007a
:1058a80061406000614060004601dd00d12c2000ad
:1058b80091407800f0cbb30000c060000240700057
:1058c800cde2b7007e0037001e0090006140600006
:1058d800c700dd00cdc2bf000074a1000140700008
:1058e800cde2b700760037001e00900061406000ee
:1058f800614060004601dd00412e200091407800a3
:10590800f0cbb30000c0600002407000e4e2b700d2
:105918006b0037001e00900061406000c700dd008a
:10592800e4c2bf000074a10001407000e4e2b700c7
:10593800630037001e009000614060006140600015
:105948004301dd00c12c20009140780070cfb300e6
:1059580000c0600002407000cce2b7005800370079
:105968001e009000614060006140600000414000fe
:10597800c12c200091407800d0cfb30000c0600057
:1059880002407000cce2b7004d0037001e009000c6
:105998006140600061416000c12e200091407800a4
:1059a800e0cfb30000c0600002407000ece2b70036
:1059b800430037001e0090006140600061406000b5
:1059c80000414000c12e200091407800d0cfb300a4
:1059d80000c0600002407000ece2b70038003700f9
:1059e8001e00900061406000614060004201dd00df
:1059f800c12e200091407800b0cfb30000c06000f5
:105a080002407000ece2b7002d0037001e00900045
:105a18006140600061416000d12c20009140780015
:105a2800e0cfb30000c0600002407000cde2b700d4
:105a3800230037001e009000614060006140600054
:105a480000414000d12c200091407800d0cfb30015
:105a580000c0600002407000cde2b70018003700b7
:105a68001e00900061406000614060004501dd005b
:105a7800c12d200091407800f0cdb30000c0600037
:105a880002407000dce2b7000d0037001e009000f5
:105a9800614060006140600000414000512f2000db
:105aa80091407800d0cfb30000c060000240700081
:105ab800f5e2b700020037009e009000b1b48800fc
:105ac8000080fa00000006000800fa00000f7800c5
:105ad800000000000000eb00b0b488001e00780051
:105ae8006101b9002207980033079800f0002000f0
:105af800010020002e019000be019000800f51008f
:105b0800818f590079003e002e009000be00900061
:105b1800006001000f003700150037001b00370038
:105b280021003700260037002c00370031003700ed
:105b3800370037003d003700410037004700370085
:105b48004d00370051003700570037005d0037001f
:105b580063003700cdc2bf000080fb004400de00b8
:105b6800614060000080fb0010079800610037006a
:105b7800cdc2bf000080fb004500de006140600030
:105b88000080fb00100798005a003700cdc2bf0004
:105b98000080fb004600de00614060000080fb00e2
:105ba8001007980053003700cdc2bf000080fb00eb
:105bb8004700de000080fb00100798004d0037000a
:105bc800e4c2bf000080fb004600de0061406000c8
:105bd8000080fb001007980046003700e4c2bf00b1
:105be8000080fb004700de000080fb0010079800e3
:105bf80040003700ccc2bf000080fb004300de003d
:105c0800614060000080fb001007980039003700f1
:105c1800ccc2bf000080fb000000d10061406000e2
:105c28000080fb001007980032003700ecc2bf006c
:105c3800614060000080fb00100798002d003700cd
:105c4800ecc2bf000080fb000000d1006140600092
:105c58000080fb001007980026003700ecc2bf0048
:105c68000080fb004200de00614060000080fb0015
:105c7800100798001f003700cdc2bf0061406000c8
:105c88000080fb00100798001a003700cdc2bf0043
:105c98000080fb000000d100614060000080fb0034
:105ca8001007980013003700dcc2bf000080fb001b
:105cb8004500de00614060000080fb00100798008e
:105cc8000c003700f5c2bf000080fb000000d100c7
:105cd800614060000080fb00100798000500370055
:105ce800b1b4800011079800020037000001eb00f2
:105cf800120798001e0090000080fa0000000600bd
:105d08000600fa002007980010002000000f780015
:105d18000000eb00100798000b0037002e009000e1
:105d28001e006000800078001e0090009efe0700a4
:105d38001e00780000004000000f78001e00900050
:105d48000000e800100798001e009000ef0f5000b8
:105d5800f2ff34000080fa00000006000600fa0096
:105d680010002000100798000000eb00000f7800da
:105d78000000eb00200798000c0037002e00900070
:105d880051ff07000000e000020032001e009000f2
:105d98001e0f40001e0090000000400010079800f1
:105da8002e0090000000e800200798002e009000c8
:105db800ef0f5000f1ff34001e0078000080fa0059
:105dc800000006000800fa00000f7800000000003c
:105dd8000000eb00b0b488001e0078006101b90033
:105de8002207980033079800f000200001002000e7
:105df8002e019000be019000800f5100818f590044
:105e080063003e002e009000be009000006001007c
:105e18000f003700150037001b003700210037003e
:105e2800270037002d0037003300370039003700ce
:105e38003f00370041003700430037004500370076
:105e480047003700490037004b0037004d00370046
:105e5800eac2bf000080fb004500de006140600030
:105e68000080fb00100798004b003700eac2bf0013
:105e78000080fb004400de00614060000080fb0001
:105e88001007980044003700eac2bf000080fb00fa
:105e98004300de00614060000080fb0010079800ae
:105ea8003d003700e2c2bf000080fb004400de0076
:105eb800614060000080fb00100798003600370042
:105ec800e2c2bf000080fb004500de0061406000c8
:105ed8000080fb00100798002f003700cbc2bf00de
:105ee8000080fb004200de00614060000080fb0093
:105ef8001007980028003700cbc2bf000080fb00c5
:105f08004300de00614060000080fb00100798003d
:105f180021003700dac2bf000080fb004600de0027
:105f2800614060000080fb00100798001a003700ed
:105f3800b1b480001107980017003700b2b4800090
:105f48001207980014003700b3b4800013079800b4
:105f580011003700b0b48000100798000e00370019
:105f6800b1b48000110798000b003700b2b480006c
:105f78001207980008003700b3b480001307980090
:105f880005003700b0b48000100798000200370001
:105f98008000eb00110798001e0090000080fa00b6
:105fa800000006000600fa00100020001007980004
:105fb8000000eb00000f78000000eb0020079800bd
:105fc8000c0037002e0090007eff07000000e00064
:105fd800020032001e0090001e0f40001e009000bc
:105fe80000004000100798002e0090000000e80014
:105ff800200798002e009000ef0f5000f1ff3400aa
:0c6008001e0078000080fa000000060076
:020000040000fa
:106014008816000006000000000000008e16000034
:10602400020000000200000000000000b81400009c
:106034008000000000000000b815000050000000bf
:10604400020000000000000000000000000000004a
:10605400000000000000000000000000000000003c
:10606400000000000000000000000000000000002c
:10607400000000000000000000000000000000001c
:10608400000000000000000000000000000000000c
:1060940000000000000000000000000000000000fc
:1060a40000000000000000000000000000000000ec
:1060b400901600000200000000000000921600008c
:1060c4000200000000000000a012000018010000ff
:1060d400000000000816000040000000000000005e
:1060e400941600000200000002000000e803000013
:1060f4000008000080080000000000009616000060
:106104000200000000000000b813000000010000bd
:106114000200000029b30900285de000185e270092
:106124006e465500c48150000b7f2a005708f300c7
:1061340060ae99003dc0110014eb07002fde35005e
:10614400d86570002c8b6d00e96c3900f0e5a00077
:10615400dbfb0f00ddf5ef0068b621008a3ba600eb
:10616400f792be001f7dbc00726156009d6a030059
:106174008e42450098b174003295f200901c1d00c7
:106184005f25020075f64100b7cef100e6830d00ed
:10619400913f6200c8b0e200059ebd003112360096
:1061a4001e78e30044305b0059fcd200b9cb8c006c
:1061b400ab9b3800a2f9c90086f44300c594f800eb
:1061c400526422005aec3300a7b2cf00c1a4e1000c
:1061d400da934f0047d9970026c6d700d47b9c009a
:1061e4004c797100fd37ff001719e700bb15480013
:1061f400d1675100230c06007a4e20003c5c0e004f
:10620400ca538000c387df00d3b554000077ad00c4
:10621400a5ea2d00d06b8800c77e8d00a3b463006f
:10622400acdc4b0073e86f00e4cced0049fe3e00ab
:106234006984160024768f00a185a9000a34ba0067
:10624400b8aa4d00cd897c00ee109f00fabf4a0029
:106254001b820400c2012e003a664000a896580032
:10626400d6afd5009a1a2b00000000004816000093
:106274004000000000000000801000002002000028
:106284000200000000000000000000000000000008
:1062940000000000000000000000000000000000fa
:1062a40000000000000000000000000000000000ea
:1062b40000000000000000000000000000000000da
:1062c40000000000000000000000000000000000ca
:1065540000000000000000000000000038150000ea
:106564008000000000000000ee180000020000009f
:1065740000000000f8170000a00000000200000066
:10658400010000000000000000000a0000000000fc
:106594000000000000640000000000000000000093
:1065a400e8030000000000000000100027000000c5
:1065b4000000000000a086000100000000000000b0
:1065c40040420f0000000000000080009698000088
:1065d400000000000000e100f505000000000000dc
:1065e40000ca9a003b00000000000000e40b5400c5
:1065f400020000000000e8007648170000000000d8
:106604000010a500d4e8000000000000a0724e00b5
:1066140018090000000040007a10f3005a0000003e
:106624000080c600a47e8d000300000000c16f003e
:10663400f2862300000000008a5d780045630100b3
:1066440000006400a7b3b600e00d000000e8890074
:106654000423c7008a000000981800002a000000e4
:1066640002000000286e75006c6c290000303100b7
:106674003233340035363700383941004243440060
:1066840045460000303132003334350036373800a7
:1066940039616200636465006600000098160000ba
:1066a4006001000002000000000000000000000083
:1066b400f03f00000000a0009999b9003f000000dd
:1066c4000040e1007a843f0000000000e04d6200d9
:1066d400503f00000000e000e2361a003f000000d6
:1066e4000080b500f8e43e0000000000a0f7c600fa
:1066f400b03e00000000a000f2d77a003e00000087
:1067040000e08e0079453e0000000000e00b2e0002
:10671400113e00000000e000df7cdb003d000000d3
:106724000000a1009cc73b0000000000004c480092
:10673400b439000000000000206ca1003700000004
:106744000000000000000000000000000000000045
:106754000000000000000000000000000000000035
:106764000000000000000000000000000000000025
:106774000000000000000000000000000000000015
:106784000000000000000000000000000000000005
:1067940000000000000000000000f0003f000000c6
:1067a4000000000000244000000000000000000081
:1067b400594000000000000000408f00400000002d
:1067c4000000000088c340000000000000006a00d0
:1067d400f84000000000000080842e00410000000a
:1067e4000000d00012634100000000000084d700c4
:1067f400974100000000000065cdcd00410000007d
:1068040000205f00a002420000000000801daf00d5
:106814001544000000004000593e290046000000d5
:106824000000000000f07f000000000000000000f5
:10683400f07f0000000000000000f0007f00000076
:106844000000000000f07f000000000000000000d5
:10685400f07f0000000000000000f0007f00000056
:106864000000000000f07f000000000000000000b5
:10687400f07f0000000000000000f0007f00000036
:10688400c21800002600000002000000c418ea003c
:1068940018000000ea180900000000000200e800e7
:1068a40018000000e81806000201000000000000c3
:1068b40000000000000006000202000000000000ca
:1068c400e81800000600000000000000f0180000b6
:1068d40002000000020000000100000000000000af
:020000040000fa
:1068e4000200fa000000eb00000f780027003700d8
:1068f4009e0178001e0078004700dd0080007800cb
:10690400402b21000080400000017800c318dd0006
:10691400402a210000804000020878001e00780010
:106924004300dd008080e800402a21008080400090
:106934000000eb00800878001e0078004300dd00b2
:10694400e4004000402a2100808040000000eb0069
:10695400800878001e0078004300dd00e600400057
:10696400402a210080804000f00720008008780041
:106974001e00780080004000403b210080804000e1
:106984000000eb00800878001e0fe80010002000d3
:106994009e0f1000d6ff3400b00020004011880084
:1069a40021e2a80020a2a9002062a9000040200042
:1069b400101188008560a9008580a900910a200033
:1069c40091407800f0c8b30000c0600001c5b30076
:1069d40001407000a9e0b700a10a200091407800ae
:1069e40080cfb30000c060000014a000aae0b7008c
:1069f4009560a8009580a900b0002000c01188000f
:106a040031e2a80030a2a9003062a90000402000b1
:106a14009011880087c0a90087e0a900310b2000ed
:106a24009140780080cfb30000c060006040b300a4
:106a3400b3e0b700310b200091407800f0c8b300f8
:106a440000c0600001c2b30001407000b3e0b700b1
:106a540097c0a80097e0a9000080fa000000060093
:106a64000a00fa0010079800210798001e00900001
:106a7400400798004e009000e10f500009003200da
:106a84004e009000e20f500006003200ae0090006d
:106a94000040eb00804878000000eb0030079800cd
:106aa4000d0037008e0707001e0090004300dd0034
:106ab40080007800402a2100680050008080400057
:106ac4002e00900083020700000f78008e07070055
:106ad4001e007800300798003e0090000080fa0005
:106ae400000006000c00fa001007980041479800c7
:106af4001e009000400798004e009000e10f5000e7
:106b0400040032004e009000e20f500008003200f2
:106b14000e00370023c2bf000080fb000000d1003c
:106b2400614060000080fb00000f7800090037001e
:106b340033c2bf000080fb000000d1006140600050
:106b44000080fb00000f78000200370010002000d6
:106b5400000f78001e00e00015003a001e009000af
:106b6400500798005e009000e10f500004003200ce
:106b74005e009000e20f5000070032000c00370066
:106b84004e4090000080fb0020118800100020007f
:106b940030079800080037004e4090000080fb004a
:106ba400a011880010002000300798000200370070
:106bb4000000eb00300798003e0090000080fa00cf
:106bc400000006000600fa0010079800210798004c
:106bd4000000eb00000f78000b0037001e00780067
:106be400800078002e009000008040001040780063
:106bf400804078001e009000baff07000000e0000b
:106c0400010032001e0fe8001e00780080007800aa
:106c14002e00900000804000104078000004e00046
:106c2400eeff3a000000eb000080fa0000000600ce
:106c34000800fa00100798001e0090003007980022
:106c44003e009000e10f5000060032003e0090002c
:106c5400e20f5000030032000000eb002007980010
:106c64000c0037001e0707001e0090004300dd00e3
:106c740080007800402a2100680050000080400015
:106c840040020700000f78001f0707001e0078006d
:106c9400200798002e0090000080fa0000000600f3
:106ca4000600fa00100798001e00900020079800c4
:106cb4002e009000e10f5000040032002e009000de
:106cc400e20f5000080032000e00370023c2bf005c
:106cd4000080fb000000d100614060000080fb00e8
:106ce400000f78000900370033c2bf000080fb00aa
:106cf4000000d100614060000080fb00000f7800bc
:106d04000200370010002000000f78001e007800f9
:106d14000080fa00000006000600fa00000f780068
:106d24001e007800200798002e009000e10f50000c
:106d3400040032002e009000e20f500008003200e0
:106d44000e0037001e00780080004000403b210008
:106d540000804000100078001007980009003700f8
:106d64001e00780080004000403b2100008040006d
:106d74001000780010079800020037000000eb00b4
:106d8400100798001e0090000080fa000000060022
:106d94000400fa00000f78001e0078001007980025
:106da4001e009000e10f5000040032001e0090000d
:106db400e20f500001003200060037001e00780088
:106dc40080004000403b2100808040000000eb0038
:106dd400800878000080fa00000006000800fa002d
:106de400100798001e009000200798002e009000c5
:106df400e10f5000040032002e009000e20f50001a
:106e0400010032001f003700b50607001e00900085
:106e14004300dd0080007800402a21006800500013
:106e240000804000cd0107001e009000300798004c
:106e34003e009000e10f5000060032003e0090003a
:106e4400e20f50000a0032000d00370030118000bc
:106e5400000f780022c2bf00614060000004e0001f
:106e6400faff3a0006003700b0118000000f7800e6
:106e740032c2bf00614060000004e000faff3a0043
:106e8400a10607000080fa00000006000400fa00d2
:106e9400000f78001e007800100798001e00900074
:106ea400e10f5000040032001e009000e20f500079
:106eb40006003200090037002342a9000000000048
:106ec4002342a80000000000040037003342a90058
:106ed400000000003342a800000000000080fa0017
:106ee40000000600809fbe000000fa0000958000ac
:106ef4001195800061004000e08048000095880002
:106f0400119588008580a9000080fa004f00be001a
:106f140000400600809fbe000000fa001400370005
:106f2400309580008000e8005095800080806000eb
:106f340040958000808f500003003a00100020002c
:106f4400a09d88000a0037002195800030958000bc
:106f540080804000301180008048780030958000a7
:106f64008000e80050958000008060003095880023
:106f740022c2bf00614060000004e000e8ff3a0064
:106f84008560a9000080fa004f00be0000400600a2
:106f9400809fbe000000fa000095800011958000db
:106fa40061004000e0804800009588001195880049
:106fb40087e0a9000080fa004f00be0000400600f0
:106fc400809fbe000000fa00140037007095800016
:106fd4008000e800909580008080600080958000ab
:106fe400808f500003003a0010002000b09d8800fc
:106ff4000a00370061958000709580008080400011
:10700400b011800080487800709580008000e8000e
:1070140090958000008060007095880032c2bf00a7
:10702400614060000004e000e8ff3a0087c0a90066
:107034000080fa004f00be00004006000400fa0081
:10704400100798001e009000000f78000800370019
:107054001e007800104078000000fb005fe5070088
:10706400804078001e007800014878001e0fe80078
:107074001e007800104078000004e000f4ff3a009d
:107084000080fa00000006000400fa0010079800cf
:107094001e009000000f7800080037001e007800e2
:1070a400104078000000fb0053e5070080407800a2
:1070b4001e007800014878001e0fe8001e007800ca
:1070c400104078000004e000f4ff3a000080fa0069
:1070d400000006000800fa00881f780010079800d6
:1070e400210798000000eb00000f78001e009000bc
:1070f400104078000004e00003003a000000eb00b8
:1071040030079800460037001e00780080007800a1
:107114002e00900000804000104078000000fb002a
:107124002ee50700000478001e0078008000780037
:107134001e00900000804000104078000000fb001a
:1071440026e50700800f5400150032002e00900041
:107154000000e800200798002e00900010407800fe
:107164000004e00003003a000000eb003007980040
:107174002b0037002e00900090407800c0c7b30069
:1071840080cf5000f1ff3a002e0090000000e8008c
:10719400200798000000eb00000f78001b00370068
:1071a4001e0fe8001e007800800078002e0090007a
:1071b40000804000104078000004e0000800320025
:1071c4001e007800800078002e00900000804000af
:1071d40090407800c0c7b30080cf50000b003a0045
:1071e4001e007800800078001e009000008040009f
:1071f40010407800520007000000e00003003a004d
:107204001e00780030079800050037007002200047
:107214009e0f1000bcff34001e0078003007980059
:107224003e0090004f0478000080fa000000060041
:107234000600fa0010079800210798000080eb0070
:10724400000f78000e0037001e00900010417800f7
:107254001e007800800078002e009000008040001e
:1072640010407800804f510005003a001e00900045
:107274000000e800100798000080eb00000f780081
:107284001e0fe8001e007800800078002e00900099
:1072940000804000104078000004e000eaff3a005b
:1072a4001e0090000080fa00000006000400fa00ae
:1072b400000f780041e429001e007800dcff07007d
:1072c400000f78001e00780090407800d0c2b30010
:1072d40080cf5000050032001e00780090407800f6
:1072e400b0c2b30080cf500001003a001e0fe80086
:1072f40071e429001e007800cdff0700000f78001c
:1073040091e429001e007800c9ff0700000f7800ef
:107314001e007800104078000004e00003003200f2
:107324000000eb0010079800020037001000200056
:10733400100798001e0090000080fa00000006006c
:107344000400fa00004f78001e00fb00b1e40700bf
:107354000000e00003003a00f0c5b3009e4f1000a7
:1073640003003a00100020001007980002003700c4
:107374000000eb00100798001e0090000080fa0047
:10738400000006000c00fa0020079800310798005e
:10739400420798000000eb00000f780041e4290048
:1073a4002e009000a2ff0700200798001e0037005f
:1073b4001e0078004200dd00800078003e0090004e
:1073c40000804000900078002e00900041ff0700ec
:1073d400100798001e0090000000e0001100320029
:1073e4001e009000800078002e0090000080400075
:1073f40041e429008eff0700200798001e00780052
:107404004200dd00800078003e00900000804000d3
:10741400900090002e009000010001005007980099
:107424000c0037001e0fe8001e0078004200dd004b
:10743400800078003e00900000804000100078003a
:10744400104078000004e000d9ff3a004e0090009c
:10745400500798005e0090000080fa0000000600cb
:107464000600fa00004f7800110798001e009000f3
:10747400440007000000e000030032000000eb00bd
:1074840020079800100037001e009000900078003c
:107494001e00900010009000008040001e487800fc
:1074a4001e009000100090008000e8001e00900074
:1074b40030009000808060001e0090001100980051
:1074c40010002000200798002e0090000080fa0091
:1074d400000006000600fa00000f7800110798006b
:1074e4001e0090003b0007000000e0000600320090
:1074f4009e0078000040eb00804878000000eb001c
:1075040020079800120037001e00900090007800b9
:107514001e00900020009000008040009040780001
:107524001e007800014878001e00900020009000a2
:107534008000e8001e009000300090008080600011
:107544001e009000210098001000200020079800e1
:107554002e0090000080fa00000006000200fa00ed
:10756400000f78009e0078000000eb00a000980057
:107574009e0078000000eb00900098000080fa0064
:10758400000006000400fa00000f78001e007800d6
:10759400100090008000e8001e0078003000900089
:1075a400808060001e00780020009000808f5000d2
:1075b40003003a0010002000100798000200370072
:1075c4000000eb00100798001e0090000080fa00f5
:1075d400000006000400fa00000f78001e00780086
:1075e400a00090001e00780010009000808f5000d2
:1075f40003003a0010002000100798000200370032
:107604000000eb00100798001e0090000080fa00b4
:10761400000006000200fa00000f78001e00780047
:10762400900090001e0078002000900080805000a0
:107634001e00780030009000008060000080fa0096
:10764400000006000600fa00000f780011079800f9
:107654001e009000460007000000e0000300320016
:107664000000eb0020079800110037001e00900076
:10767400900078001e009000100090000000400070
:10768400008040001e0878001e009000100090004a
:107694008000e8001e0090003000900080806000b0
:1076a4001e00900011009800100020002007980090
:1076b4002e0090000080fa00000006000600fa0088
:1076c400000f7800110798001e0090003c0007008e
:1076d4000000e000060032009e0078000000eb008d
:1076e400800878000000eb002007980013003700a2
:1076f4001e009000900078001e0090002000900072
:107704000000400000804000900078001e007800d7
:10771400010878001e009000200090008000e8001e
:107724001e00900030009000808060001e009000d9
:107734002100980010002000200798002e009000df
:107744000080fa00000006000200fa00000f780032
:107754009e0078000000eb00a00098009e007800d6
:107764000000eb00900098000080fa000000060082
:107774000400fa00000f78001e007800100090004a
:107784008000e8001e0078003000900080806000d7
:107794001e00780020009000808f500003003a0003
:1077a4001000200010079800020037000000eb00d2
:1077b400100798001e0090000080fa0000000600e8
:1077c4000400fa00000f78001e007800a00090006a
:1077d4001e00780010009000808f500003003a00d3
:1077e4001000200010079800020037000000eb0092
:1077f400100798001e0090000080fa0000000600a8
:107804000200fa00000f78001e007800900090003b
:107814001e00780020009000808050001e00780038
:1078240030009000008060000080fa000000060034
:107834008a00fa000000eb0020079800c982a90022
:10784400c9a2a900c9c2a900c9e2a900cd82a900a0
:1078540000000000cda2a90000000000cdc2a900d4
:1078640000000000cde2a90000000000416a2000f1
:107874009140780000ccb30000c060003040b300f9
:10788400a4e6b700416c20009140780000ccb3001e
:1078940000c060003040b300c4e6b700616a200055
:1078a4009140780000ccb30000c06000b040b30049
:1078b400a6e6b700c16c20009140780000ccb3006c
:1078c40000c060005040b300cce6b700816a2000dd
:1078d4009140780000ccb30000c060005041b30078
:1078e400a8e6b700a16d20009140780000ccb30059
:1078f40000c060007040b300dae6b700316d2000cc
:107904009140780000ccb30000c060000034a000b7
:10791400d3e6b700f522a80000000000f122a90078
:1079240000000000eefb070094010700b40007000c
:107934006d0207007ff50700e600470020da290002
:10794400801f7800b0da2900801f780070db2900de
:10795400801f780001007800f4e70700e6875700ed
:10796400e60047002000200096fc07006007200086
:107974000e0040009f010700600720000e00400039
:10798400e6010700000820000e00400099010700ee
:10799400000820000e004000e0010700000037004e
:1079a40070b48000e10f500005003a000000eb00c5
:1079b40070b48800600720000e004000d701070063
:1079c40070b48000e20f500005003a000000eb00a4
:1079d40070b48800600720000e004000e501070035
:1079e400660047003b0007000000e00003003a0087
:1079f4003000200010079800100037006600470090
:107a040041de29000afe0700000f78001e007800fe
:107a1400104078000004e00003003a002000200039
:107a240010079800050037004200200061c72900b4
:107a34001e00780053fe0700100798001e009000f7
:107a4400e30f5000150032001e0090000000e0001b
:107a54000f0032001e009000e20f50000c003200b4
:107a6400600520000e0040009e009000811f7800f9
:107a740071de2900811f7800ace70700e487570016
:107a8400610520008e804000200020004dfc07008e
:107a940021df2900200020004afc070060072000a5
:107aa4000e0040005f0107000001be00a0b480008a
:107ab400cf80de00800f5100818f5900b8ff36005f
:107ac400600720000e0040004a010700bdf60700d1
:107ad400b3ff37000800fa00300798000000eb00fd
:107ae40010079800e400470020002000dcfb07009a
:107af4000000e0003f003200ce4090002000200053
:107b0400f8fb07004e409000ed4f500003003a0090
:107b1400a1c0b30020002000f2fb07004e409000fb
:107b2400ed4f50001a0032004e409000e84f5000d4
:107b34000d00320081b48000f0042000808f5000da
:107b440009003c0082b480004e40900080407800e0
:107b5400805b210000004100014878000200e80039
:107b640080b488000600370080b480000000e00084
:107b74000300340080b480000000e90080b4880071
:107b8400be0090000040eb008048780019003700e8
:107b9400100020001007980081b48000805b210051
:107ba400808040000040eb00804878000000eb003b
:107bb400000f78000a0037001e007800800078006b
:107bc4003e009000008140009e007800805b210010
:107bd4000080400010407800004978001e0fe80043
:107be40080b480009e0f1000f3ff34000000eb000f
:107bf40080b488001e0090000080fa000000060097
:107c04000000fa004342a80042a2a8002124200058
:107c14009140780030ceb30000c060008041b300d2
:107c240042e2b70042c2bf003040b30042e2b700b4
:107c34004402a90041e2a8000080fa000000060006
:107c44000400fa00100798000000eb00000f780011
:107c54001e0090004012880040c2bf0061406000d6
:107c64000004e000fcff32000100370000000000c7
:107c74001e0fe800300120009e0f1000fbff3400af
:107c8400401280000080fa00000006000200fa00a2
:107c9400000f78001e00e00002003200f522a80068
:107ca40001003700f522a900000000000080fa005e
:107cb400000006001400fa00000f9800110f98004d
:107cc4000000eb00100798000000eb00000f7800a4
:107cd4000000eb00300798000f00370000c02100bf
:107ce40010079800be0090000e089000008040002d
:107cf400104078008080fb001e00900001004000ce
:107d0400100798001e009000cdff07003e00900071
:107d14000000e80030079800be0090001e089000a4
:107d2400808f5000edff3900f0ff2100c4ff0700f1
:107d34000000eb003007980004003700000000004a
:107d44003e0090000000e80030079800be0090005c
:107d540070382100808f5000f8ff36000000eb00df
:107d6400200798000000eb0030079800230037003c
:107d74000080210010079800be009000f03f200012
:107d8400808060001e0090000100400010079800f1
:107d94001e009000aaff0700000f78001e00780064
:107da4001ce207000000e00008003a001e00780012
:107db40026e207000000e00004003a001e007800fc
:107dc40034e207000000e000090032002e019000b8
:107dd4001e0078008040780080602100000041008f
:107de400014878002e0090000000e8002007980069
:107df4003e0090000000e80030079800be009000ac
:107e0400f0032000808f5000d9ff3600ae009000b0
:107e140080602100808040000040eb0080487800b2
:107e2400816021002000200066fb07000080fa002a
:107e3400000006000a00fa002007980031079800a5
:107e44003e009000e10f5000060032003e0090001a
:107e5400e20f5000030032000000eb0040079800de
:107e6400140037003e0090004a00dd00100798001f
:107e7400ae009000f03f2000808060001e00900063
:107e84000100400010079800100020007fff070049
:107e94001e0090006aff07000000eb0068ff070067
:107ea400000f78000000eb0078ff07001e00780048
:107eb400400798004e0090000080fa000000060081
:107ec4000600fa00100798002107980000c020005f
:107ed400000f78009e009000f03f200000806000ba
:107ee4001e0f40001000200068ff07001e007800ed
:107ef40053ff07002e00900051ff07000000eb0025
:107f040062ff07000080fa00000006000600fa0085
:107f140010079800210798001e009000e10f500000
:107f2400140032001e009000e20f500011003200d5
:107f34001e009000e30f500001003a000d003700ce
:107f44001e0090004a00dd00000f7800ae00900093
:107f5400f03f2000008060001e0f40001000200051
:107f64004aff07001e00780035ff07000000eb0001
:107f740046ff07000080fa00000006000000fa0037
:107f84000000eb00800888000000eb003008880047
:107f9400f07f24006008880084e0a90094e0a80031
:107fa40011e1a8000080fa00000006000000fa00b9
:107fb400b30007000080fa00000006000200fa0087
:107fc400000f78001e007800100078000080fa008e
:107fd400000006000200fa00000f78001e0078007e
:107fe400640007001e007800020007000080fa0009
:107ff400000006000200fa00000f78001e0178005d
:108004006000b80030019800410198009600070014
:108014001e01780010019800210198000080fa00e8
:10802400000006000600fa00200798008e000700f2
:10803400008fbe002e009000100078000000e000c9
:10804400230032002e009000a00090001000900049
:10805400be0f5000ae8f58000f0036002e00900067
:1080640030019000c00190002e009000a00090000c
:10807400100090003e024000ae8248000400be00a2
:1080840002004000838048002e01900030019800d7
:10809400410198000e0037002e009000300190003e
:1080a400c00190002e009000a000900010009000ed
:1080b4003e021000ae8218000400be000200400020
:1080c400838048002e0190003001980041019800ff
:1080d4002e0090001e01be0012009800230098009c
:1080e4002e00900030039000c003900086007800ba
:1080f400a0002000000ab8006030b9000501780033
:10810400000141006a38b900000141008202780090
:108114000400be000080fa00000006000200fa001d
:10812400000f78001e007800beff07009e00780054
:1081340010002000800878001e00780030039000b2
:10814400c003900086007800a0002000000ab80058
:108154006030b90005017800000141006a38b900b7
:1081640000014100820278000400be000080fa0091
:10817400000006000200fa00000f78001e007800dc
:10818400a8ff07009e0078000000eb00800878003c
:108194001e00780030039000c00390008600780031
:1081a400a0002000000ab8006030b9000501780082
:1081b400000141006a38b9000001410082027800e0
:1081c4000400be000080fa00000006000600fa0069
:1081d40020079800240007000001be002e00900034
:1081e40001002000001f4100019749001e00070004
:1081f400be0f5000ae8f5800fcff39000080fa001b
:10820400000006000600fa00200798001600070088
:10821400008fbe002e009000e90f500008003600c9
:108224002e009000a2002000110009000280d80056
:10823400010020001e0f40005e9748000400370034
:1082440010002000010020001e0f40005e9748002f
:1082540005000700be0f5000ae8f5800fcff390028
:108264000080fa00000006000000fa000400070085
:1082740050b4800061b480000080fa000000060061
:108284000200fa0042b4800050b4800061b480005f
:10829400000f51001e0078006101b80050b4800046
:1082a40061b48000020040008380480050b488001c
:1082b40061b488000080fa0000000600801f780086
:1082c4000000fa000000eb003008880040b4800091
:1082d4000000e80040b4880084e0a9000080fa00af
:1082e4004f007800004006000000fa000208200059
:1082f400f10f200080532100dde507000080fa0023
:10830400000006001000fa0060479800410798003a
:10831400224f9800334f98006e4090000080fb007d
:108324004300de000080fb00200798006e409000b0
:108334008080fb002e0090004300dd000080500090
:1083440067001000100798006e4090000080fb004a
:108354000000d1000080fb00000f78006e40900008
:108364000080fb00800040000008210000804000e5
:10837400ce009000010878001e0078007007980075
:108384006e4090000080fb000000a20061006000cd
:108394000004e0000e0032009e00780080532100ab
:1083a40000804000104078006f4160002e4890002b
:1083b4000080fb004400dd008040780000cfb30063
:1083c40000c0600000404100404f98000b0037009f
:1083d4009e00780080532100008040001040780007
:1083e4008040780000cfb30080c060002e48900029
:1083f4006f40600000c04000404f9800805321004f
:10840400fe00900000804000ce48900001487800b3
:108414003e4890000080fb0060004000e10f5000e7
:108424000f003e00ae019000ae0090000028210035
:108434000080400010407800004178003e489000e1
:108444008080fb001e0090000008dd0000406900f1
:108454008040780000282100008041000148780015
:108464000080fa00000006001000fa00604798003f
:108474004107980052079800630798006e409000e7
:108484000080fb004300de000080fb002007980012
:108494006e4090008080fb002e0090004300dd00c1
:1084a4000080500067001000100798006e40900094
:1084b4000080fb000000d1000080fb00000f78006a
:1084c4004e0090000000e000080032006e40900072
:1084d4000080fb0080004000000821000080400074
:1084e400900078004e009000010878005e00900033
:1084f4000000e0001b0032009e0078008053210041
:1085040000804000904078005e00900001487800b0
:108514006e4090000080fb000000a200610060003b
:108524000004e000080032005e0090001040780073
:108534008080fb00000f2000008060004480de008b
:10854400604f9800040037005e00900010407800ef
:108554006f406000604f98005e009000ee4890000d
:10856400014878006e0090000000e0000a0032002c
:10857400ae009000002821000080400010407800e8
:108584008080fb001e0090000088de00e140600057
:108594006e009000014878000080fa000000060098
:1085a4000000fa00021020008000eb000008210007
:1085b4002fe50700020220008000eb0000282100c4
:1085c4002be5070002082000f10f20008053210052
:1085d40027e507000080fa00000006000a00fa0000
:1085e4001007980041479800320798001e00900039
:1085f4000000e000030032003e0090000000e000b4
:1086040003003a00100020004007980034003700af
:108614001e009000bfe40700000f78009e80e80071
:10862400f00f2000808f500003003600100020005f
:10863400400798002a0037003e009000e700400001
:108644003e009000704092000080fb0000804000db
:108654009e0090000de507003e009000f04092005f
:108664001e00780080c040003e00900071409a00d7
:108674003e009000e70040003e00900070409200f1
:108684000080fb00808040000040eb0080487800c0
:108694003e009000704092008040e8003e00900050
:1086a40071409a003e009000e70040003e009000b8
:1086b400704092000080fb00808040004e4090009b
:1086c400804878003e009000704092008040e800ae
:1086d4003e00900071409a000000eb0040079800b3
:1086e4004e0090000080fa00000006000e00fa0020
:1086f400500798000000eb00300798005e009000df
:108704000000e000580032005e0090001040780045
:108714000080fb00801f780080df2900801f780024
:108724008064210081e40700e4875700816421000c
:108734002000200023f907005e0090000000e800fc
:10874400801f780080e02900801f78008064210069
:1087540076e40700e48757008164210020002000ac
:1087640018f9070081e129002000200015f907000d
:108774000000eb0040079800350037005e009000d1
:10878400e70040003e009000008040001007980081
:1087940091c0b30020002000d2f807009e00900092
:1087a4002000200007f907001e00900059e407008c
:1087b400800078003e0090000100400030079800df
:1087c4003e0090000000e800300798003e00900052
:1087d400de00900066004000010040001040900060
:1087e4000000fb00200798003e0090000000e80015
:1087f400300798002e009000600798006e009000eb
:108804000000e000080032006e009000e10f50000c
:108814000100320008003700a1e2290020002000f6
:10882400e8f807000700370041e329002000200092
:10883400e4f8070003003700f1e3290020002000da
:10884400e0f807004e0090000000e80040079800a0
:108854005e009000604090008080fb004e0090001d
:10886400808f5000c5ff3e000080fa000000060023
:108874000800fa0020079800310798000040eb0038
:10888400204798000000eb00000f78000d0037002f
:108894002e4090000081fb009e0078002e00900086
:1088a40000804000104078000000fb008000690058
:1088b400803b2100008040009040780021479800d0
:1088c4001e0fe8003e0090009e0f1000f0ff3900dc
:1088d4002e4090000080fb000080fa00000006009b
:1088e4000000fa0090b480000000e00001003a00ab
:1088f400ff3ffc0090b480000000e80090b48800c2
:108904000080fa00000006000000fa0090b4800025
:108914000000e90090b4880090b480000000e000fa
:1089240001003a000000fc000080fa00000006008c
:00000001FF
